:100000000C9425050C945D050C945D050C945D0520
:100010000C945D050C945D050C945D050C945D05D8
:100020000C945D050C945D050C94FC170C94D51D87
:100030000C9407290C945D050C945D050C945D05EA
:100040000C945D050C945D050C945D050C945D05A8
:100050000C945D050C94D5180C945D050C945D050D
:100060000C945D050C945D050C945D050C945D0588
:100070000C945D050C945D050C945D050C945D0578
:100080000C945D050C945D050C945D050C945D0568
:100090000C945D050C945D050C945D050C945D0558
:1000A0000C945D050C945D050C945D050501090239
:1000B000A10185020901A100050919012905150001
:1000C00025019505750181029501750381010501E1
:1000D000093009311581257F950275088106093897
:1000E0001581257F950175088106050C0A380215D2
:1000F00081257F950175088106C0C005010980A191
:1001000001850319012AB700150126B7009501756D
:10011000108100C0050C0901A101850419012AA064
:1001200002150126A002950175108100C005010984
:1001300006A1018506050719E029E71500250195A7
:1001400008750181020507190029EF1500250195A1
:10015000F0750181020508190129059505750191C0
:1001600002950175039101C00660FF0961A10109B3
:1001700062150026FF0095207508810209631500AD
:1001800026FF00952075089102C005010906A1010E
:10019000050719E029E71500250195087501810279
:1001A0009501750881010507190029FF150026FF33
:1001B0000095067508810005081901290595057542
:1001C000019102950175039101C00000000000003B
:1001D000000000000000000000000000000000001F
:1001E00000000000000000000000000000007E0F82
:1001F00000D4FFFFFFC700000078000000000000EF
:1002000000002A2B28000000000000000000000071
:10021000000000000029000000002C1E34202122D4
:1002200024342627252E362D3738271E1F2021223D
:10023000232425263333362E37381F0405060708B6
:10024000090A0B0C0D0E0F101112131415161718A6
:10025000191A1B1C1D2F3130232D350405060708E4
:10026000090A0B0C0D0E0F10111213141516171886
:10027000191A1B1C1D2F3130354CFD377A585A0086
:100280000004E6D6B4460200210116000000742FD7
:10029000E5A3E00433016B5D003D8889C65436C395
:1002A000174FE4E338EFF14B8CD99458D8A104B63A
:1002B00026E280DE778D9E37BD3AA9CBBA292B770F
:1002C00015A89699FC0E99A90139921AABBEBEE108
:1002D000BBC27955F3C864B3111C530D46CC221927
:1002E00025745CF78E258A4E5FC9C7DD294166708B
:1002F000EE6E96A00B1EE5202FD85AD05FDAC27B97
:10030000BEE37D1243C0D5EEE8FACA8ABEDFF89894
:10031000FEDA35514AE85C1F90DD8B2A0B3FB6F5BB
:1003200015383EB36E00D9B4F6989DEE2C8B07932A
:100330008F25ECF52FA780BFFDEF14DCC84EA486F7
:10034000D830E44A1EC4DEE35C7517937EEDEF16E9
:10035000C9CDFA89A4E4F72E5DDFAF1B44302EEB44
:10036000EDFE587E33112EB331C0622B60A568229A
:10037000A82B69CED0BDFEDE28FCD8855599323F2A
:100380003805B923BCD08B8AB70FDECBFF7D8E2317
:10039000BD127CE4F4A9954E015627E718F2E97ED8
:1003A000C622ABD4F527C14FE8B7419B3FCBAFC9BD
:1003B000BB72F8F2593A7FEF12BD8CAC82432BD15D
:1003C000202FE1B499917B810254DE4D023BDA3853
:1003D000908262E784B35AF0776CD98BD182FC02A9
:1003E0007D4424C73CDC41D84C1684CE6214CFA88F
:1003F000EB2977E17677CC143C9FB5A8BEE0DD957C
:10040000B6BF6F00000052D18FBE13E1FC3900016E
:100410008703B40800001802431BB1C467FB020045
:1004200000000004595A000000000200010006000C
:1004300002000C0003000D0004000E0005000F0078
:10044000060011000700130008001400090017003F
:100450000A0018000B001F000C0020000D002100F6
:100460000E0023000F00270010002A0011000001D9
:100470000101010101010101020202020202020264
:100480000203030303030303030404040404040436
:1004900005050505050606060606070707070708FA
:1004A000080808090909090A0A0A0B0B0B0C0C0CAD
:1004B0000D0D0D0E0E0E0F0F0F1010111111121247
:1004C00013131414151516161717181819191A1AC4
:1004D0001B1B1C1D1D1E1E1F202021222223242425
:1004E000252626272829292A2B2C2D2D2E2F303161
:1004F0003232333435363738393A3B3C3D3E3F4073
:100500004142434445464748494A4C4D4E4F50515D
:100510005354555658595A5B5D5E5F616264656617
:1005200068696B6C6D6F7072737577787A7B7D7E9E
:100530008082838587888A8C8E8F91939596989AEE
:100540009C9EA0A2A3A5A7A9ABADAFB1B3B5B7BA06
:10055000BCBEC0C2C4C6C9CBCDCFD1D4D6D8DBDDDA
:10056000DFE2E4E7E9EBEEF0F3F5F8FAFDFF002651
:100570003646002737470028384800293949002ADD
:100580003A4A002B3B4B01263646012737470128C4
:10059000384801293949012A3A4A012B3B4B0226A6
:1005A00036460227374702283848007464540075DD
:1005B00065550076665600796959007A6A5A007B5B
:1005C0006B5B01746454017565550176665601795B
:1005D0006959017A6A5A017B6B5B02746454027533
:1005E00065550276665600A4948400A5958500A6FC
:1005F000968600A7978700A8988800A99989027B0A
:100600006B5B01A4948401A5958501A6968601A73C
:10061000978701A8988801A9998902796959027A6E
:100620006A5A002E3E4E002F3F4F0030405000319E
:100630004151003242520033435301AC9C8C012E95
:100640003E4E012F3F4F01304050013141510132A8
:1006500042520133435302A7978702A89888007C2F
:100660006C5C007D6D5D007E6E5E0081716100825C
:1006700072620083736301AD9D8D017C6C5C017DB2
:100680006D5D017E6E5E0181716101827262018326
:10069000736302A9998900AC9C8C00AD9D8D00AE5E
:1006A0009E8E00AF9F8F00B0A09000B1A19101AECF
:1006B0009E8E01AF9F8F01B0A09001B1A191022940
:1006C0003949022A3A4A022B3B4B29003A003B00A7
:1006D0003C003D003E003F0040004100420043001E
:1006E000440045004C00460035001E001F0020005D
:1006F00021002200000023002400250026002700FE
:100700002D002E002A002B0014001A0008001500EE
:1007100017004B001C0018000C00120013002F00E3
:1007200030003100390004001600070009000A00FB
:100730002A000B000D000E000F00330034002800CB
:100740004E00E1001D001B000600190005002800F6
:1007500011001000360037003800E500520000009C
:10076000E000E300E20000002C00E000E1002C00CB
:100770000000E6000151E400500051004F00005C11
:100780000100010001000100010001000100010061
:10079000B200B300AF00B100145CDE5C01000100E8
:1007A0000100010001000100000001000100010042
:1007B00001000100010001005300C25CC35CC95C80
:1007C000C55C010001004A000100010001000100B8
:1007D00001000100010001000100CC5CCA5CCB5C9F
:1007E0000100010001000100010001000100010001
:1007F000010001004D0001000100010001000100A5
:100800000100010001000100010001000100A80039
:10081000A90000000100010001000000010001002A
:1008200001000100000001000100AE00AC00AA00C0
:10083000AB00010001000100010001000100010006
:1008400001000100010001000100010001000100A0
:100850000100010001000100010001000000010091
:100860000100010001000100010001000100010080
:100870000100010001000100010001000100010070
:100880000100010001000100010001000100010060
:100890000100010001000100010001000100010050
:1008A0000100010001000100010001000100010040
:1008B0000100010001000100010001000100010030
:1008C0000100010001000000010001000100000022
:1008D0000100010001000100000001000100010011
:1008E0000100010001000100010001000100010000
:1008F00001000100010001000100010001000100F0
:1009000001000100010001000100010001000100DF
:1009100000000100010001000100010001000100D0
:1009200001000100010001000100010001000100BF
:1009300001000100010001000100010001000100AF
:10094000010001000100010001000100010001009F
:10095000010001000100010001000100010001008F
:10096000010001000100010001000100010001007F
:100970000100010001000100010000000100010070
:100980000100000001000100010001000000010061
:100990000100010001000100010009025B000301E8
:1009A00000A0FA090400000103010100092111015E
:1009B000000122400007058103080001090401002D
:1009C0000203000000092111010001222200070595
:1009D000820320000107050303200001090402002F
:1009E000010300000009211101000122BC000705DC
:1009F0008403200001120100020000000842586137
:100A00004E0100010203011C037600690061006CC5
:100A1000003A0066003600340063003200620033A2
:100A200000630000000E034E0041005400550052C8
:100A300000450000000E0358002D0042004F0057F3
:100A40000053000000040309040011241FBECFEF6F
:100A5000DAE0DEBFCDBF04B603FE18C080916C069D
:100A600090916D06A0916E06B0916F068730904B05
:100A7000A740B04B59F410926C0610926D0610927C
:100A80006E0610926F06E0E0F8E3099526E0AEED01
:100A9000B2E001C01D92AC36B207E1F712E0A0E06F
:100AA000B1E0E2ECF5E602C005900D92AE3DB10773
:100AB000D9F70E942E290C94A9320C940000E8ED7D
:100AC000F0E080818E7F80831092E2001092DA0045
:100AD0001092E100A0EEB0E08C9181608C93808157
:100AE0008F77808319BCA7EDB0E08C918E7F8C93BB
:100AF00080818F7E80831092060608952091E40005
:100B00003091E50095E6A9012091EC00822F8170DB
:100B100020FF06C08091E80080FF06C080E00895B5
:100B20002091E80022FD1AC080913406882389F0C4
:100B3000853089F08091EB0085FD0FC02091E400A5
:100B40003091E50042175307F9F29150E1F684E045
:100B5000089582E0089583E0089581E00895EF927A
:100B6000FF920F931F93CF937C018B010E947E0510
:100B7000C82F811117C08091E80085FD0BC08091BE
:100B8000E8008E778093E8000E947E05882399F321
:100B9000C82F08C0F70181917F018093F1000150B7
:100BA000110949F78C2FCF911F910F91FF90EF9072
:100BB0000895CF93FC0180913406843001F5C091F3
:100BC000E900CF702091EC00922F917020FD90E809
:100BD000C92B82E08093E9008091E80080FF0CC07F
:100BE00050E040E060E270E0CF010E94AF058091EC
:100BF000E8008E778093E800CF70C093E900CF9132
:100C0000089580912C0687FF13C08091E80082FF31
:100C100006C08091E8008B778093E80004C0809143
:100C200034068111F2CF0895809134068823D9F3D8
:100C30008091E80080FFF8CF8091E8008E77ECCFBC
:100C4000982F9093E900242F762F50E0891731F0E8
:100C50007091EC002091ED005091F00021FD07C053
:100C60009F5F973071F78093E90081E0089530919C
:100C7000EB003E7F3093EB003091ED003D7F3093F1
:100C8000ED003091EB0031603093EB007093EC009D
:100C90002093ED005093F0002091EE0027FDE0CF6F
:100CA00080E00895B0E0A0E0E8E5F6E00C940831BB
:100CB000C8EDD0E088818F7E8883E7EDF0E0808109
:100CC0008160808384E082BF81E080930606888112
:100CD0008E7F888302EE10E0F80110821092DA0015
:100CE00081EEC82ED12CF601108288818F778883FF
:100CF00088818068888388818F7D888319BC109261
:100D0000340610922B0610922A061092290690EEB5
:100D1000E92EF12CF70180818B7F808388818160AF
:100D2000888342E060E080E00E942006F601808136
:100D30008E7F8083F80180818160808380818860DC
:100D40008083F70180818E7F8083888180618883A2
:100D5000CDB7DEB7E8E00C942431FC018091320677
:100D60009091330686179707A0F06115710529F455
:100D70009091E8009E779093E80090E061157105EE
:100D800051F4911108C08091E80082FF34C080E0E6
:100D90000895BC01F2CF809134068823C1F18530DB
:100DA000C1F18091E80083FD30C08091E80082FDB0
:100DB000EACF8091E80080FFE1CF8091F30020919D
:100DC000F200382F6115710519F02830310558F0FF
:100DD00091E02830310509F090E02091E8002E776D
:100DE0002093E800CBCF81918093F100615071098D
:100DF0002F5F3F4FE7CF80913406882341F0853045
:100E000041F08091E80083FFBECF81E0089582E049
:100E1000089583E00895089580910806089520912B
:100E200013012223C9F02091010627FF15C0E62FE8
:100E3000E695E695E695EE31D8F4E80FF92FF11D29
:100E4000677021E030E001C0220F6A95EAF7209533
:100E50008281282322830895FC01329608962191ED
:100E6000621303C0DF0111971C92E817F907B9F765
:100E70000895209113012223C1F02091010627FF3C
:100E800014C0E62FE695E695E695EE31F8F4E80F06
:100E9000F92FF11D677021E030E001C0220F6A9543
:100EA000EAF78281822B82830895FC0132962FEF2C
:100EB00030E04191641751F02F3F19F4411101C006
:100EC000232F3F5F3630A9F72F3F09F40895820F93
:100ED000911D27FD9A95FC01628308952091FA05E2
:100EE0003091FB052817390771F09093FB0580932B
:100EF000FA05E091F805F091F905309721F00084AA
:100F0000F185E02D099508952091F6053091F705BA
:100F10002817390771F09093F7058093F605E09153
:100F2000F805F091F905309721F00680F781E02D62
:100F300009950895E091F805F091F905309729F0A9
:100F40000190F081E02D0995089580E00895FA015F
:100F5000811101C0FB0109950895EDE3F6E02481BC
:100F600030E1231B08F420E024838091EF038160AB
:100F70008093EF030895EDE3F6E0248130E1230F41
:100F800008F42FEF24838091EF0381608093EF03B7
:100F9000089590913D06937071F080933E066093A2
:100FA0003F06493C08F048EC409340068091EF032F
:100FB000822B8093EF030895EDE3F6E0438120E177
:100FC000421B08F440E0818121E0628190E00E94B0
:100FD000C9070895EDE3F6E0438120E1420F08F4EC
:100FE0004FEF818121E0628190E00E94C90708955E
:100FF000EDE3F6E0628120E1621B08F460E08181AC
:1010000021E0438190E00E94C9070895EDE3F6E0F6
:10101000628120E1620F08F46FEF818121E043815A
:1010200090E00E94C9070895EDE3F6E0818121E098
:10103000438162818850990B0E94C9070895EDE3AE
:10104000F6E0818190E021E04381628108960E9470
:10105000C907089590913D06937061F081110BC00E
:10106000946090933D06109212018091EF03862BBD
:101070008093EF030895823110F09464F2CF880FCB
:10108000880F982BEECF80913D06869586958150EE
:1010900009F481E161E00E942A08089580913D06EB
:1010A000869586958F5F823108F081E061E00E942D
:1010B0002A0808958093110180913D0683708093E2
:1010C00010010E94E41283E0809312010895EF92D0
:1010D000FF920F939701201B31092F3F310519F023
:1010E00010F02FEF30E02095382F320F08F43FEF4B
:1010F000832F0F91FF90EF900895EF92FF920F933F
:101100009701201B31092F3F310519F010F02FEF07
:1011100030E0322F3095482F430F08F44FEF842FE3
:10112000620F0F91FF90EF900895EF92FF920F934F
:101130001F930E0D1F2D111DF90137FF03C0F195EF
:10114000E195F10924E0EE0FFF1F2A95E1F7EF3F4B
:10115000F10519F014F0EFEFF0E09A0157FF03C02A
:1011600031952195310994E0220F331F9A95E1F7CB
:101170002E173F070CF4F901E00FF11FEF3FF105C7
:1011800019F010F0EFEFF0E0E095282F3E2F230F3D
:1011900008F42FEF822F1F910F91FF90EF90089589
:1011A000EF92FF920F93970195E0099F200D311D5B
:1011B00011242F3F310519F010F02FEF30E020956A
:1011C000382F320F08F43FEF832F0F91FF90EF90ED
:1011D000089522E8241B08F420E0620F089540954A
:1011E000282F429F412D1124842F0895EF920F93B1
:1011F000972F23E0029FB0011124759567956E0D1E
:10120000792F0F91EF900895E42FF0E0EE0FFF1F7C
:10121000E652FE4F6081621B0895E42FF0E0EE0F6E
:10122000FF1FE752FE4F6081621B0895622F0895F1
:101230000E94B31308950E94751308950F931F938E
:1012400010E0F801EE0FFF1FE752FE4F90819C5512
:1012500097FD9195000F111FF801E652FE4F008196
:101260000152110B2003F001219FF00D112408E31E
:1012700010E0091B110997FD139540039001419F50
:10128000300D1124E20FF31F9F01220F331F2E0F89
:101290003F1F37FF02C021583F4F220F232F221F2D
:1012A000330B620F1F910F910895FC019B01009772
:1012B00029F480E077FF2BC080E80895AC0197FF08
:1012C00004C044275527481B590BB901640F751FEB
:1012D00037FD10C0241B350BC901A5E0880F991FED
:1012E000AA95E1F70E94353180E2861BF7FF0FC017
:1012F00081950895CB0165E0880F991F6A95E1F704
:10130000BA01621B730B0E94353180E6EECF08955F
:10131000EF920F93CF93DF93D72FC82FC9010E19E8
:10132000BA010E945509602F681B7D2F8C2FDF9119
:10133000CF910F91EF900895EF920F931F93CF935A
:10134000DF93D62FC72F182FC9010E19010FBA012D
:101350000E945509081B202F219F212D1124822F27
:101360006D2F7C2FDF91CF911F910F91EF900895FA
:101370000F93CF93DF93D72FC82FC901BA010E94D3
:101380005509682F600F7D2F8C2FDF91CF910F9122
:101390000895E82F86FDE0952E2F2F7086FD2F5F94
:1013A000E695E695E695E670F0E0E859FE4F918106
:1013B000929F902D212D112492959F702295207F30
:1013C000922B2081920F87FD919580E8890F0895D7
:1013D000AC018230910508F408959FEF413E8EE103
:1013E000580740F49A0195E0369527959A95E1F7CC
:1013F00098E0920F61E0E62FE90FFF27FF1F9F01A2
:1014000035952795822F229FF001239FF00DF00D37
:1014100011244E175F0738F49FEF920F961758F775
:101420008FEF860F08952F3FE9F361E0620FF6CF4B
:1014300030E020E0869F212D969F200D311D112444
:10144000C9010895AF92BF92CF92DF92FF920F939E
:101450001F93CF93DF93362F472FE82FF0E0E25909
:10146000FB4F71110FC0E4918E2F2E2F6E2F722F14
:10147000DF91CF911F910F91FF90DF90CF90BF90A0
:10148000AF900895C72FD0E02491F22E022F10E0E4
:1014900056E0659FC0011124EFEFF0E0BF010E940C
:1014A000EA30832F90E0880F991F35E5369FD001F1
:1014B000379FB00D11248A1B9B0B982F990F980F03
:1014C0006F01CC1ADD0AC09ED001C19EB00DD09E26
:1014D000B00D11248B2F499FA0011124452F5527B2
:1014E0006F01C41AD50AC09EA001C19E500DD09EA6
:1014F000500D11245F01A91AB108AC9E6001AD9E88
:10150000D00CBC9ED00C1124CD2CDD24EC19FD098F
:10151000E09FE001E19FD00DF09FD00D1124ED2F51
:1015200062307105A1F050F46115710509F49ECF88
:101530006130710581F0EB2F852F98CF64307105F4
:1015400069F080F06630710509F490CFF4CFE22F96
:101550002B2F8D2F8BCFE22F252F88CFEB2F822F94
:101560002D2F84CF2B2F8F2DE52F80CF2F923F92C1
:101570005F926F927F928F929F92AF92BF92CF9223
:10158000DF92EF92FF920F931F93CF93DF93CDB72C
:10159000DEB72A970FB6F894DEBF0FBECDBF8B83A0
:1015A0007E836D832091140182E1289F802D112478
:1015B0008F838E5E89838A83883510F037E53A837E
:1015C000809143068C83FF81EF2FF0E0FA87E98753
:1015D000CF01880F991F9C0127523E4F69013B8123
:1015E000832F90E0FC013196F887EF838A819985FB
:1015F0009817E8F081E0E981E73508F080E02A9665
:101600000FB6F894DEBF0FBECDBFDF91CF911F9113
:101610000F91FF90EF90DF90CF90BF90AF909F9091
:101620008F907F906F905F903F902F900895E98505
:10163000FA85E957FD4F8081909115018923F1F0DA
:1016400020903E0630903F062F8138852D5B394F24
:1016500039015B8010E0FC815F16D0F020914006DC
:10166000129F112D1124B101812F0E94220A462FB1
:10167000282F672F89859A850E941B0929853A851D
:101680002F5F3F4F3A87298732E0C30ED11CAECF80
:10169000F30181913F01F601A080A81ABB08818067
:1016A000F3018781881A9908AA9C9001AB9C300DA0
:1016B000300D1124889CC001899C900D900D11243F
:1016C000820F931F0E94E809082F6091410621E0D4
:1016D000620F08F46FEFF301EE0FFF1FE354F640C3
:1016E000858996890E94180A7C019401A501B1019F
:1016F000812FED81FE8109951B015394182FABCFEB
:10170000B0E0A0E0E6E8FBE00C9408318C01C09169
:10171000140182E1C89FC02D112422E1D22EDC0EDB
:10172000CD2C27E52D1510F497E5C92E2091410603
:1017300031E0230F08F42FEF30E050E040E06FEF8E
:101740007FEF80E090E00E9446327901D0E02C2FBC
:10175000CC1550F081E0F6E5FD1508F480E0CDB73A
:10176000DEB7E8E00C942431FE01E957FD4F80819B
:1017700090911501892311F1409143064150042EA7
:10178000000C550B47FF1CC0C7016091410621E0CA
:10179000620F08F46FEF0E94180AAC0160913E06D8
:1017A00070913F0680914006F80109950E94220A37
:1017B000462F282F672FCE010E941B092196C7CFE5
:1017C000FA01ED5BF94F818982130AC0FA01EE0F2D
:1017D000FF1FED5BF94F818D928D8E159F05A8F24D
:1017E00041505109CFCFB0E0A0E0E9EFFBE00C940D
:1017F00003315C01C091140182E1C89FC02D112406
:1018000012E11C0FF12E183510F037E5F32E609120
:10181000410666958091390690913A060E94180A11
:10182000782ED0E0CF1548F081E0173508F080E041
:10183000CDB7DEB7EDE00C941F31FE01E957FD4F47
:101840008081909115018923C9F1CE01880F991FDC
:1018500081589E4FFC01E65AFF4F2081422F4C5584
:10186000550B6A01855A9F4FFC018081282F215218
:10187000330B4901449F9001459F300D300D1124D9
:10188000889CC001899C900D900D1124820F931F9C
:101890000E94E809082F60913E0670913F068091F2
:1018A0004006E72C9401A601F50109950E94220A41
:1018B000462F282F672FCE010E941B092196B2CFF9
:1018C000B0E0A0E0E6E6FCE00C9409317C01C091B8
:1018D000140182E1C89FC02D112412E11C0F012FB9
:1018E000183508F007E5609141066695669521E098
:1018F000620F08F46FEF8091390690913A060E94CA
:10190000180AD82ED0E0C01748F081E0173508F04B
:1019100080E0CDB7DEB7E7E00C942531FE01E95752
:10192000FD4F808190911501892391F060913E06D1
:1019300070913F06809140062D2D4C2FF70109959F
:101940000E94220A462F282F672FCE010E941B09D2
:101950002196D9CF9091BD03803F59F48091BE0369
:1019600087FF0DC01092BE0391110BC01092B503FA
:1019700008C0813F81F48091BE0318169CF399231F
:1019800081F08091BF039091C003892B09F064C05E
:101990001092B4030895823F49F497FFF0CF10925C
:1019A000BD038091BE038111ECCFE0CF833F19F4DA
:1019B0001916ACF3E4CF2091BF03893F29F4121626
:1019C000F4F61092BF03DBCF8A3F19F427FFD7CF7D
:1019D000F8CF2091C0038B3F29F427FFD0CF10927E
:1019E000C003CDCF8C3F19F41216CCF3C8CF843F7F
:1019F00031F48091BC038E7F8093BC03C0CF853FC0
:101A000021F48091BC038D7FF7CF863F21F4809134
:101A1000BC038B7FF1CF873F21F48091BC03877F8C
:101A2000EBCF883F21F48091BC038F7EE5CF8D3FC3
:101A300031F48091B6038E7F8093B603A0CF8E3FA2
:101A400021F48091B6038D7FF7CF8F3F09F097CFB8
:101A50008091B6038B7FF0CF08958091B60380FD0F
:101A600016C081FD16C082FD16C08091B403882384
:101A7000A1F0883280F428E0829FC001112468E23E
:101A800070E00E943531862F672B39F0089582E08F
:101A9000089584E0089588E0089581E00895809194
:101AA000B60380FD14C081FD14C082FD16C0809174
:101AB000B503882381F08E3180F420E5829FC00138
:101AC00011246EE170E00E943531862F089584E183
:101AD000089588E2089588E0089580E50895803F9C
:101AE00031F40E944F0D81958093BE030895813F8C
:101AF00019F40E944F0DF8CF823F31F40E944F0D30
:101B000081958093BD030895833F19F40E944F0D82
:101B1000F8CF893F29F40E942D0D8093BF030895CB
:101B20008A3F21F40E942D0D8195F7CF8B3F31F430
:101B30000E942D0D81958093C00308958C3F19F468
:101B40000E942D0DF8CF843F31F48091BC03816059
:101B50008093BC030895853F21F48091BC0382608B
:101B6000F7CF863F21F48091BC038460F1CF873F9B
:101B700021F48091BC038860EBCF883F21F48091F1
:101B8000BC038061E5CF8D3F31F48091B603816065
:101B90008093B60308958E3F21F48091B60382604E
:101BA000F7CF8F3FB9F78091B6038460F1CF80E023
:101BB0000895F894E82FE295EF70F0E031A1282F16
:101BC0002F7081E090E001C0880F2A95EAF7982FE6
:101BD0009095932391A392A1892B82A37894089541
:101BE0009091010692FF06C0282F28712830F9F441
:101BF000877F846093FF06C0282F28712831F1F475
:101C0000877E84612091020620FF06C0382F38713C
:101C10003830D9F4877F816021FF06C0282F2871D2
:101C20002831D1F4877E816194FD877E0895282F25
:101C300024712430F9F68B7F8860DCCF282F247143
:101C4000243101F78B7E8861DDCF382F317131303F
:101C500019F78E7F8860E0CF282F2171213121F77D
:101C60008E7E8861E1CFCF93DF93EC0182389105BE
:101C7000A9F1D8F58133910509F496C048F5893268
:101C8000910509F48AC08A9709F495C0C11521E528
:101C9000D20708F0BCC0C11530E5D30708F014C165
:101CA000C83ED10508F09CC0C03ED10560F5C83AD9
:101CB000D10508F087C0C53AD10508F0FDC0C13094
:101CC000D10509F12097F9F0C430D105E0F440C006
:101CD0008533910509F45AC0C997C1F68091010670
:101CE000837089F0C0EED0E00EC0833E910599F17B
:101CF00070F4803E910501F1823E910539F68091A4
:101D0000010682FD21C0CE01DF91CF910895863E6C
:101D1000910561F1873E910571F1843E910509F0CD
:101D2000B5CF8091020681FFEECF80910106C7EE0C
:101D3000D0E084FD0DC0E7CF8091010680FD12C187
:101D40009091020690FFDFCFC3EED0E084FFDBCF9F
:101D5000D0E0C0E0D8CF8091010682FD06C190910D
:101D6000020690FDBFCF84FFCECFF2CF8091010657
:101D700083FDDDCFC8CF8091010683FDF9C090912E
:101D8000020691FFF0CFC4EED0E0BDCF80910106F6
:101D900085FFB9CFC9E2D0E0B6CF8091010685FFBB
:101DA000B2CFC5E3D0E0AFCF8091010686FFABCFC5
:101DB000CAE2D0E0A8CF8091010686FFA4CFC1E39C
:101DC000D0E0A1CFCF3BD10518F6C85AD0E0CC0F58
:101DD000DD1FCB5DDE4F0990D881C02DD46493CF39
:101DE000C11540E2D40758F4C11581E0D80708F0C6
:101DF0008ACFC03FD10508F4ABCFD06584CFC115E1
:101E000090E4D90708F4A4CFDF70D06A7CCFC11565
:101E100025E5D20700F5C11534E5D30708F08AC0DF
:101E2000C11543E5D40708F071C0C11582E5D80794
:101E300008F467C0CE018370992721E030E002C02A
:101E4000220F331F8A95E2F7C695C69580E2C89F98
:101E5000E001112452C0C11599E5D907A8F4C115B4
:101E600028E5D20708F06BC0C11536E5D30708F0A6
:101E70006FCF8C2F0E94F00DC82FD0E0DC2FCC2725
:101E8000CC27DF71D0623FCFC1154AE5D40708F4F3
:101E90005BC0CE0190568115904208F059CF8D2F2E
:101EA0008F710E94F00D90E0982F882788279F71EE
:101EB0009C012C2BE901E6CFC55AD0E0CE5DDE4F68
:101EC000C881D0E0D0641FCFCE01E4E0969587951D
:101ED000EA95E1F783702C2F26952695237040E232
:101EE000249F90011124382B8C2F8370C1E0D0E007
:101EF00002C0CC0FDD1F8A95E2F7C22BD32BDC6822
:101F000002CFDC2FCC27C16FD06AFDCECE0183700B
:101F1000992721E030E002C0220F331F8A95E2F7B3
:101F2000C695C69590E2C99FE0011124C22BD32B20
:101F3000DA68E9CEDC2FCC27C46FD06AE4CEDC2F80
:101F4000CC27C06FD06ADFCE8C2F8F700E94F00D2F
:101F500034E0D695C7953A95E1F7CF709C2FEC0108
:101F6000D069D1CEC9E3D0E0CECEC2EED0E0CBCEA8
:101F7000C6EED0E0C8CE80918503882331F0109260
:101F800085031092840310928303089580959091A5
:101F90008203982390938203089510926003109215
:101FA0005F0310925E03089580915D0390912C036E
:101FB000981301C008958F5F8770FACF292F96304C
:101FC00078F58F3068F590E03FE0239F800D911DFC
:101FD0001124682F677023E0969587952A95E1F77D
:101FE000FC01EE0FFF1FE80FF91FEE5FFC4F50E002
:101FF00040E080E0219130E0062E02C03695279522
:102000000A94E2F721703327042E01C0220F0A94AC
:10201000EAF7822B4F5F5F4F4330510559F7089520
:1020200080E00895292F963098F58F3088F590E05C
:102030003FE0239F800D911D1124282F277041E040
:1020400001C0440F2A95EAF723E0969587952A95D3
:10205000E1F7FC01EE0FFF1FE80FF91FEE5FFC4FE9
:1020600030E020E070E05191DF011197CB01022EAA
:1020700002C0969587950A94E2F78170819585272D
:10208000842385278C932F5F3F4F2330310559F7E9
:1020900008959C013A9521153F4150F5FC01EE272A
:1020A000F170BC0166277270AC01442754709C012A
:1020B0002227387094FF0EC080E1EF2B09F480E0F6
:1020C000672B09F08062452B09F08064232B89F08F
:1020D0008068089581E0EF2B09F480E0672B09F018
:1020E0008260452B09F08460232B19F088600895E5
:1020F00080E00895809303067093050660930406BC
:10210000809134068430F9F48093E9008FEF909148
:10211000E800815095FD06C095ED9A95F1F7000015
:102120008111F5CF8091E80085FF0DC050E040E0BF
:1021300063E070E083E096E00E94AF058091E800E4
:102140008E778093E8000895BC0184E00E947A10A5
:102150000895BC0183E00E947A1008959C0184E0F8
:102160008093E9009FEF8091E800915085FD06C0C3
:1021700085ED8A95F1F700009111F5CF8091E80087
:1021800085FF0CC050E040E066E070E0C9010E94AD
:10219000AF058091E8008E778093E8000895CF9393
:1021A000DF93EC01809113018823B1F18091010646
:1021B00087FF32C060E284E08093E9008FEF909166
:1021C000E800815095FD06C095ED9A95F1F7000065
:1021D0008111F5CF8091E80085FF1BC0809113012C
:1021E00070E050E040E0811104C050E040E068E061
:1021F00070E0CE010E94AF058091E8008E77809359
:10220000E80080E2FE01A9E0B6E001900D928A9517
:10221000E1F7DF91CF91089568E081E0CDCF81E0D3
:102220008093E00080E28093D8001092C9008FE193
:102230009EE40197F1F700C0000087E090EBDC011D
:1022400080936C0690936D06A0936E06B0936F0614
:1022500088E19CE00FB6F894A895809360000FBECB
:1022600090936000FFCFCF93DF93C7EFD2E060E0A1
:10227000CE010E9422322196C11584E0D807B9F719
:10228000DF91CF9108951F93CF93DF93122F843066
:10229000E0F46630D0F44F30C0F4C42FD0E0CC0F5F
:1022A000DD1F9EE1699FC00DD11D112494EB899F14
:1022B000C00DD11D1124632FCE0187960E942232BA
:1022C000612FCE0188960E942232DF91CF911F911B
:1022D00008958F929F92AF92BF92CF92DF92EF922A
:1022E000FF921F93CF93DF938090F0059090F105BC
:1022F00081E090E09093F1058093F0058AECC82E80
:1023000086E0D82ED0E07601C0E014C0F50125911A
:102310003491412F6C2F8D2F0E94431182E0A80E23
:10232000B11C1F5F1F3091F78EE1E80EF11CCF5FEB
:10233000C63019F0570110E0E9CFDF5F84EBC80E1B
:10234000D11CD43001F79092F1058092F005DF9115
:10235000CF911F91FF90EF90DF90CF90BF90AF9003
:102360009F908F900895CF93C82F6FEF81116FEAE0
:1023700083E290E00E9422326FEFC11168E284E2B2
:1023800090E00E9422326FEFC11162ED85E290E091
:102390000E942232CF91089580E00E94B31160E044
:1023A00086E290E00E9422320E9469110E9433115D
:1023B00081E00E94B31108950F931F93CF93DF9391
:1023C000843030F5663020F54F3010F5C42FD0E062
:1023D000CC0FDD1F2EE1629FC00DD11D112434EB07
:1023E000839FC00DD11D1124CE0187960E94043217
:1023F000082F10E0102F0027CE0188960E9404328B
:102400009801282BC901DF91CF911F910F91089559
:1024100090E080E0F8CF462F2091F4053091F5054B
:10242000232B99F4703F39F4603F79F48091F205E1
:102430009091F3050895843040F4763030F46F3095
:1024400020F4672F0E94DC11089590E080E0089549
:10245000CF92DF92FF920F931F93CF93DF936C0184
:102460000091380680918603082BC7E0D0E010E089
:10247000FC2EC8010C2E02C0959587950A94E2F7B0
:1024800080FD0CC02197A0F7F12C8F2DDF91CF910B
:102490001F910F91FF90DF90CF900895B6018C2F80
:1024A0000E940B120E94330E019761F3EECFCF937F
:1024B000DF93EC010E942812BE010E940B120E94C1
:1024C000330EDF91CF910895FC01808191810E94AC
:1024D000571292959F70963091F058F4925F9F70CA
:1024E000923058F4803F19F030F4883E30F481E0A7
:1024F00008959A5FF4CF843FD1F380E00895883E39
:10250000B0F3813FD1F7F3CF83E290E00E94043231
:102510008F3A89F484E290E00E940432883259F4C0
:1025200085E290E00E94043291E0823D09F090E063
:10253000892F8170089580E0FCCFCF9384E090E0F4
:102540000E940432C82F82E290E00E940432982F49
:102550008C2FCF910895EF92FF920F931F93CF93FB
:10256000DF93062F10E00C541A4FF8019081992345
:1025700021F1E82EEE0CF0E96F9FE0011124CC5F11
:10258000DB4F84E2F82EF092F003E1EFF3E0DE019E
:102590008D91819384E0E130F807D1F724E630E0B3
:1025A00041E150E060EF73E08E2D0E94C930E0E120
:1025B000FE0E6096F4EBFF12E6CFF8011082CDB765
:1025C000DEB7E6E00C94263160E084E70E94AB12AF
:1025D00061E086E70E94AB1262E085E70E94AB12E1
:1025E0000895E0EFF3E06083418324E630E042E0C9
:1025F00050E0BF01880F0E94C9300895EF92FF920A
:102600000F931F93CF93DF93E82E062F10E0035113
:102610001A4FF8018081882381F0F2E16F9FE00179
:102620001124C954DA4FF12C49916F2D8E2D0E943F
:10263000F112F39482E1F812F7CFF8011082CDB7CE
:10264000DEB7E6E00C942631CF93DF93C82F4BE042
:102650006DEF0E94F11240E06AE08C2F0E94F112AF
:102660008FE39CE90197F1F700C0000040E060E0D3
:102670008C2F0E94F11240E061E08C2F0E94F11239
:1026800040E066E08C2F0E94F11240E06DEF8C2F4D
:102690000E94F112D0E040E06D2F8C2F0E94F112C9
:1026A000DF5FD231C1F740E06D2F8C2F0E94F11215
:1026B000DF5FD432C1F740E06D2F8C2F0E94F11202
:1026C000DF5FD43BC1F74BE06DEF8C2F0E94F1121E
:1026D00041E06AE08C2F0E94F11240E06DEF8C2FF8
:1026E0000E94F112DF91CF910895A4E0B0E0EBE7F2
:1026F000F3E10C940B31F62E042F122F8735910540
:1027000070F5880F991F880F991FBC0162597A4F85
:1027100044E050E0CE0101960E94CE318981837061
:10272000EA81282F30E040E9849FC00111248C5FAA
:102730009B4FE80FF92FF11DB497F082EB81E80F62
:10274000F92FF11DB4970083EC81E80FF92FF11DEB
:10275000B49710832C543A4F81E0F901808324967A
:10276000E5E00C942731FF920F931F93CF93DF93F3
:10277000182F062FF42ED0E0C0E02F2D402F612F10
:10278000CE010E9475132196C735D105B1F7CDB79B
:10279000DEB7E5E00C942731A4E0B0E0E2EDF3E130
:1027A0000C9402310E94263084E70E94241386E7AD
:1027B0000E94241385E70E9424130EE615E052E1DF
:1027C000752E68E0C62ED12CEE24E394F12C6624FD
:1027D000639444E050E0B801CE0101960E94CE31EE
:1027E0004A8150E0CA0184972B81622F6452770B93
:1027F0004B012C81E22FE452FF0B5F0129812370F2
:1028000030E0FC0197FD379643E0F595E7954A9552
:10281000E1F7729EA001739E500D112449545A4F46
:10282000E40FF52FF11DB6010E943531A70101C05B
:10283000440F8A95EAF78081842B8083F40197FC0A
:10284000379693E0F595E7959A95E1F7729EC0016A
:10285000739E900D112489549A4FE80FF92FF11DA2
:10286000C401B6010E943531A70101C0440F8A9509
:10287000EAF78081842B8083F501B7FC379683E0EB
:10288000F595E7958A95E1F7729EC001739E900DCC
:10289000112489549A4FE80FF92FF11DC501B60193
:1028A0000E943531A70101C0440F8A95EAF7808163
:1028B000842B808323513A4FF90160820C5F1F4FB4
:1028C000F6E00A3C1F0709F084CF60E084E70E942D
:1028D000FE1261E086E70E94FE1262E085E70E9438
:1028E000FE122496EEE00C941E31B0E0A0E0EBE77F
:1028F000F4E10C9409318C01FC01E957FD4F808112
:10290000682349F1D0903F06D0914006C0913E0621
:10291000EC2EF12C0E94BE31282FC7018C549F4F02
:1029200068E671E00E9435318E199F0997FD039684
:10293000959587959595879523706C2F289F600DA9
:1029400011247D2D8D2F0E94220A462F282F672FBC
:10295000C8010E941B09CDB7DEB7E7E00C94253112
:10296000B0E0A0E0E6EBF4E10C940631182F809182
:102970001101811323C090913D06937020911001A5
:1029800030E081E09217130609F480E081708093B3
:1029900016018091420690911501981739F08093A5
:1029A000150140E060E080E00E941809123160F4F7
:1029B000E12FF0E0E555FD4C0C94493181E0E6CF84
:1029C00080911601811102C0C0E0B0C040E060E01B
:1029D00080E00E941809F8CFC091140182E1C89FDD
:1029E000C02D112402E10C0FF02E083510F0F7E590
:1029F000FF2E60913E0670913F06809140060E9436
:102A0000220AE62ED72EC82ED0E0CF1528F0C1E03E
:102A1000073508F48BC0D8CFFE01E957FD4F808100
:102A200090911501892331F02C2D4E2D6D2DCE0165
:102A30000E941B092196E9CFC091140182E1C89F31
:102A4000C02D112402E10C0FF02E083510F0E7E53F
:102A5000FE2EE0903E06D0913F06D0904006609159
:102A600041066695669566958091390690913A067D
:102A70000E94180A0E94C909805887FD8195880F15
:102A8000382F2D2D329F312D1124832F6E2D7D2F28
:102A90000E94220AE62ED72EC82ED0E0CF1508F0CD
:102AA000B6CFFE01E957FD4F808190911501892332
:102AB00031F02C2D4E2D6D2DCE010E941B0921963B
:102AC000EDCF8CE999E00E94F30B04C086E199E018
:102AD0000E94600CC82F2AC08DE099E0F9CF84E0F5
:102AE00099E0F6CF86EF98E0EECFC091140182E135
:102AF000C89FC02D112472E1F72EFC0EEF2C87E544
:102B00008F1510F467E5E62E609141066695809179
:102B1000390690913A060E94180AD82ED0E0CE15B8
:102B2000E8F0C1E026E52F1508F44ECF809114019E
:102B30008F5F80931401C1110CC082E08093120159
:102B400080911601811105C0111103C083E08093AB
:102B50001201CDB7DEB7EAE00C942231FE01E9574D
:102B6000FD4F808190911501892311F1CE01880FCD
:102B7000991F81589E4FFC01E55AFF4F2081215239
:102B8000330B865A9F4FFC0140814C55550B609189
:102B90003E0670913F06809140060D2D0E94B809B7
:102BA0000E94220A462F282F672FCE010E941B0960
:102BB0002196B5CF88E899E086CFC091140182E1D3
:102BC000C89FC02D112442E1F42EFC0ECF2C37E516
:102BD0003F1510F437E5C32E609141066695669562
:102BE0008091390690913A060E94180AD82E80E406
:102BF0008D0D0E94C90990E8B92EB80E8D2D0E9446
:102C0000C90920E8A22EA80ED0E0CC1530F0C1E012
:102C1000E6E5EF1508F08ACFD7CEFE01E957FD4F64
:102C20008081909115018923A1F060913E067091F9
:102C30003F0680914006ED2C0C2F2A2D4B2D0E9433
:102C40001E090E94220A462F282F672FCE010E94BC
:102C50001B092196DACFC0911601C1111EC06091E7
:102C6000410620E1620F08F46FEF809139069091E0
:102C70003A060E94180A6AE070E00E94EA30892B46
:102C800009F0A2CE0E94BE3167E570E00E943531A6
:102C9000609115010E94751449CFC091140182E121
:102CA000C89FC02D112402E10C0F802F083508F0B9
:102CB00087E5D0E0E82EF12CCE15DF050CF0A7CE8D
:102CC00060911501CE010E9475142196F5CF8FEE0B
:102CD00098E00E94800BFECE89EE98E0FACF8091BA
:102CE000430621E0382F321B08F430E0832F60EDDB
:102CF00078E00E94B60AEECE8091430621E0382F9C
:102D0000321B08F430E0832F65E978E0F2CF809140
:102D1000430621E0382F321B08F430E0832F6DE7A3
:102D200078E0E7CF67E678E080E0E3CF46E050E088
:102D30006CE170E08DE396E00E9412321092EF0396
:102D400008958F929F92AF92BF92CF92DF92EF92AF
:102D5000FF921F93CF93DF938091EA039091EB034F
:102D6000A091EC03B091ED032FB7F8948090FD058E
:102D70009090FE05A090FF05B09000062FBF750152
:102D80006401C81AD90AEA0AFB0A2FB7F8944091DD
:102D9000FD055091FE056091FF05709100062FBF63
:102DA0004093EA035093EB036093EC037093ED03BD
:102DB0001091C103E1ECF3E0C12FD0E00197AF4FD8
:102DC000BF4F88199909AA09BB091D1327C0C093D1
:102DD000C1038091EE03C0E0811108C080913D06DF
:102DE000C82FC37019F0C82FC695C69580911201DF
:102DF0008130F1F1882329F1823009F44AC083300F
:102E000009F44BC0DF91CF911F91FF90EF90DF90BD
:102E1000CF90BF90AF909F908F900895218D328D6D
:102E20004901B12CA12C88159905AA05BB0520F4F0
:102E3000C150DF5F3296C9CF2C0D3D1D328F218FDF
:102E4000F8CF109214014093390650933A066093DC
:102E50003B0670933C0689E2E1ECF3E0A3E4B6E0C4
:102E600001900D928A95E1F781E080931201CACF1B
:102E70008C2F0E94B014CC2329F20E949A0781FF64
:102E8000C1CF2FEF4FEF6FEF8DE290E00E941B0953
:102E9000B9CF8C2F0E945A08B5CF8091EF038111D2
:102EA0000E9496164091390650913A0660913B0671
:102EB00070913C062FB7F8948091FD059091FE0526
:102EC000A091FF05B09100062FBF841B950BA60BA8
:102ED000B70B4097A105B10508F494CF10921201E9
:102EE00091CFEDE3F6E085E1808380911701909129
:102EF0001801A091190181839283A3838FE78483B2
:102F00008FEF85830E949616089590E080E00E94DE
:102F10000C32883E9E4F19F40E948412089580E07E
:102F2000089568EE7EEF90E080E00E94403260E01D
:102F300082E090E00E94223260E083E090E00E9414
:102F400022321092860360E084E090E00E942232F8
:102F500064E082E290E00E94223260E085E090E04E
:102F60000E94223260E086E090E00E9422326FEF01
:102F700087E090E00E94223240E050E0BA0188E011
:102F800090E00E94343260E08DE090E00E942232B6
:102F900040E050E0BA0188E190E00E94343260E005
:102FA00087E190E00E94223240E050E0BA018CE1DB
:102FB00090E00E94343270E060E080E290E00E9495
:102FC000403240E050E0BA0188E190E00E943432A3
:102FD00080E00E94B3110E94CC1140E050E0BA01A1
:102FE0008FE090E00E94343240E050E0BA0183E18B
:102FF00090E00E94343208951F920F920FB60F9204
:1030000011242F933F934F935F936F937F938F93ED
:103010009F93AF93BF93EF93FF938091E10082FF63
:1030200009C08091E20082FF05C08091E1008B7FA2
:103030008093E1008091DA0080FF24C08091D80065
:1030400080FF20C08091DA008E7F8093DA0080912B
:10305000D90080FF9DC080E189BD82E189BD09B4AE
:1030600000FEFDCF81E08093340680910606811139
:1030700009C00E945F050E9452068091E2008460B0
:103080008093E2008091E10080FF17C08091E20010
:1030900080FF13C08091E2008E7F8093E2008091D8
:1030A000E20080618093E2008091D800806280938A
:1030B000D80019BC85E0809334068091E10084FF3C
:1030C0002BC08091E20084FF27C080E189BD82E1AE
:1030D00089BD89B5982F917080FFFBCF8091D80072
:1030E0008F7D8093D8008091E1008F7E8093E100F6
:1030F0008091E2008F7E8093E2008091E200816007
:103100008093E20080912B06882309F447C084E075
:1031100080933406809134068091E10083FF27C0BC
:103120008091E20083FF23C08091E100877F80933C
:10313000E10082E08093340610922B068091E1003A
:103140008E7F8093E1008091E2008E7F8093E20089
:103150008091E20080618093E20042E060E080E0E4
:103160000E9420068091F00088608093F000FF911B
:10317000EF91BF91AF919F918F917F916F915F91EF
:103180004F913F912F910F900FBE0F901F90189568
:1031900019BC109234061092060674CF8091E30099
:1031A00087FD93E090933406B5CF78941F921FB6B5
:1031B0001F9211248F939F93AF93BF938091FD052E
:1031C0009091FE05A091FF05B09100060196A11D0A
:1031D000B11D8093FD059093FE05A093FF05B0936C
:1031E0000006BF91AF919F918F911F901FBE1F90BE
:1031F00018959C014FB7F8948091FD059091FE05BC
:10320000A091FF05B09100064FBF821B930B08955C
:103210002FB7F8948091FD059091FE05A091FF05D0
:10322000B09100062FBF08950E9408199C0190914B
:10323000BD038091BE03982B21F03093BA032093F5
:10324000B9039091BF038091C003982B21F0309374
:10325000B8032093B703E091F805F091F905309792
:1032600049F082E08093BB030480F581E02D8BEB75
:1032700093E009950895ACE0B0E0E1E4F9E10C9445
:1032800004318E010F5F1F4F8CE0F80111928A9577
:10329000E9F793E5E92E91E0F92E6801AA24A394B9
:1032A000B12CF70181917F018F3F09F446C0F8945A
:1032B000E82FE295EF70F0E021A18F70A50102C028
:1032C000440F551F8A95E2F7CA01922F982B91A3BC
:1032D00092A18095892382A3789400C0E9E5F1E06A
:1032E00021E030E0912C812C41914F3F09F489C0BD
:1032F000A42FA295AF70B0E090968C9190E04F70A3
:1033000002C0959587954A95E2F780FD7AC0C9017C
:10331000882A992A220F331F51E0E836F50721F752
:10332000F701319780818F3F11F00E94D90D80EA1B
:103330008A95F1F7F60191828082F2E0CF0ED11CDE
:1033400049E5E41641E0F40609F0ABCF4CE050E06B
:10335000B8018AE893E00E94D731FF24F3940097E4
:1033600009F4F12C892B09F44FC08CE0F801AAE88C
:10337000B3E001900D928A95E1F781E08093890393
:103380000E94081990938803809387038091870394
:10339000909188030E94F9180397D0F180918A03D5
:1033A00090918B039093A9038093A80380918C0341
:1033B00090918D039093AB038093AA0380918E0329
:1033C00090918F039093AD038093AC038091900311
:1033D000909191039093AF038093AE0380919203F9
:1033E000909193039093B1038093B00380919403E1
:1033F000909195039093B3038093B2031092890345
:1034000007C090E080E084CF809189038111BECF16
:103410008F2D2C96ECE00C942031809182039091BA
:103420008103892B8093E00280918503882329F111
:103430000E9408192091830330918403821B930B0F
:103440008838934110F00E94BB0F8091E002909168
:103450008503892B8093E002809113018823E1F199
:103460008091010687FF38C08EE1E2EEF2E090E045
:103470008150A0F591110E94BB0F40E250E061E63F
:1034800073E080EE92E00E94D731892B21F180E237
:10349000E0EEF2E0A1E6B3E001900D928A95E1F74B
:1034A000E091F805F091F9053097A9F080911301AA
:1034B000882359F08091010687FF07C08091E002C0
:1034C0008093E10286E08093E0020280F381E02DA8
:1034D00080EE92E00995089586E0C7CF21912223DE
:1034E00039F29F5FC5CF90E080E00E94840790E0B2
:1034F00080E00E946E07109281030E940D1A86E000
:10350000EBEBF3E0DF011D928A95E9F71092B5032A
:103510001092B4031092B6030E9414190895809378
:1035200038060E94731A089580913806982F967075
:10353000963021F488600E948F1A0895877FFBCF10
:1035400021E030E001C0220F8A95EAF720958091B2
:10355000380682230E948F1A089590916003809507
:10356000892380936003282F277091F4282F082E39
:10357000000C330B9217130659F09091020692FF3C
:1035800007C08595859585950E94A01A0E94CD0F4C
:103590000895CF93C0910206C2FB992790F998171E
:1035A00091F080FBC2F9C09302066091010684E0AD
:1035B00090E00E9422326C2F82E290E00E94223240
:1035C00082E00E94AD1ACF91089521E030E001C061
:1035D000220F8A95EAF780913806822B0E948F1A73
:1035E0000895809386030E94731A089510928203AF
:1035F00080911301E2EEF2E0882361F080910106F0
:1036000087FF08C08EE1DF011D928A95E9F70E94CD
:10361000731A089586E0F7CFAAE2B0E0E2E1FBE199
:103620000C940D318CE296E02091F100DC012D9399
:10363000CD01B6E084339B07B9F780912D06833026
:1036400009F472C0B8F4813009F449C0823009F439
:10365000B3C08091E80083FF96C280912C069091C0
:103660002D069A3008F08FC2E92FF0E0E354FD4CAC
:103670000C9449318A3009F48EC08B3009F471C042
:10368000893039F780912C06813219F78091300604
:1036900090913106009711F00297D9F68091E800D9
:1036A000877F8093E8008091E80082FF38C0909186
:1036B000F3008091F200029731F48091F1008130A3
:1036C00011F0863021F48091F100809308068091FA
:1036D000E8008B778093E8000E940106BACF8091C2
:1036E0002C06813A09F0B5CF8091E800877F80935E
:1036F000E8008091300690913106892B61F460E2F8
:1037000089E096E070E00E94AD068091E8008B773A
:103710008093E8009ECF60E090E080E0F3CF80915E
:1037200034068111C0CF95CF80912C06813A09F0E3
:1037300090CF8091300690913106892B09F089CF86
:103740008091E800877F8093E8008091E80080FF07
:10375000FCCF809113018093F1008091E8008E7777
:10376000B9CF80912C06813209F073CF8091300659
:1037700090913106892B09F06CCF8091E800877F0A
:103780008093E8000E94010680912E068093130129
:103790000E94F61A5ECF80912C06813209F059CF33
:1037A0008091E800877F8093E8000E940106809165
:1037B0002F06809307064DCF80912C06813A09F0A1
:1037C00048CF8091E800877F8093E8008091E800EF
:1037D00080FFFCCF80910706BECF803899F08238F9
:1037E00009F0D1C1809130068F70873008F0CBC1CD
:1037F0008093E9008091EB0085FB882780F9109287
:10380000E90006C08091290690912A0691118260F4
:103810009091E800977F9093E8008093F1001092D8
:10382000F1008091E8008E77AAC1882309F498C13D
:10383000823009F0A8C180912E0681119BC1809130
:1038400030068F702FEF280F263008F09CC1809330
:10385000E9002091EB0020FF8DC1933031F480917D
:10386000EB0080628093EB0085C19091EB0090614A
:103870009093EB0021E030E001C0220F8A95EAF737
:103880002093EA001092EA008091EB008860EACF72
:10389000811179C110912E061F778091E300807805
:1038A000812B8093E3008091E800877F8093E8007C
:1038B0000E9401068091E80080FFFCCF8091E30028
:1038C00080688093E30082E0111183E080933406E6
:1038D0005AC18058823008F056C120912E0630918E
:1038E0002F062C3DE3E03E07A1F583E08A838AE2C0
:1038F00089834FB7F894DE01139620E03EE051E251
:10390000E32FF0E050935700E49120FF03C0E295CD
:10391000EF703F5FEF708E2F90E0EA30C0F0C796F7
:103920008D939D932F5F243159F74FBF8091E8000D
:10393000877F8093E8006AE270E0CE0101960E94E2
:10394000AD068091E8008B778093E8001CC1C0969B
:10395000E7CF8091300690913106432F55274330B1
:10396000510509F44AC078F54130510509F485C084
:103970008BE590E0EAE9F9E04230510509F003C136
:103980002091E800277F2093E800209132063091B3
:1039900033068217930708F49C0140E02115310596
:1039A00009F070C041116EC08091E80082FDC9CF5E
:1039B00080913406882329F2853019F28091E8003D
:1039C00083FFF2CFBECF4132510509F447C04232E6
:1039D000510509F0D8C08330910508F0D4C0FC012E
:1039E000EE0FFF1FED58FE4F0190F081E02D805942
:1039F0009E4FDC018C9190E01DC0332721303105B2
:103A0000E9F02115310579F022303105F9F0233044
:103A1000310509F0B8C0E7E0FAE0E4918E2F90E0BC
:103A2000E7E0FAE007C0E5E4FAE0E4918E2F90E0E9
:103A3000E5E4FAE0009709F4A6C0A2CFE5E3FAE0D6
:103A4000E4918E2F90E0E5E3FAE0F4CFE5E2FAE0CE
:103A5000E4918E2F90E0E5E2FAE0ECCF833091051F
:103A600008F091C0880F991FFC01E758FE4F0190A4
:103A7000F081E02D89E090E083CF82E190E0E5EFF6
:103A8000F9E07ECF80913406882309F45ACF85303F
:103A900009F457CF8091E80083FD53CF8091E8006F
:103AA00082FD82CF8091E80080FF78CF9091F30073
:103AB0008091F2002115310519F08830910550F000
:103AC00041E0089709F040E08091E8008E7780930C
:103AD000E80064CF44914093F100319621503109C0
:103AE0000196E8CF803809F04EC08091E800877FCA
:103AF0008093E80080912B068093F10092CE811193
:103B000042C010912E061230F0F58091E800877FB8
:103B10008093E80010932B060E940106112311F0F8
:103B200084E005C08091E30087FDFACF81E08093B7
:103B3000340642E061EC81E00E94200642E261EC42
:103B400084E00E94200642E261EC82E00E942006AE
:103B500042E260EC83E00E9420068091340613C0AC
:103B600080912E06813079F481E0933009F080E075
:103B700080932A061092E9008091E800877F809365
:103B8000E8000E9401068091E80083FF0AC080914E
:103B9000E800877F8093E8008091EB00806280934B
:103BA000EB00AA96E3E00C9429311F920F920FB616
:103BB0000F9211242F933F934F935F936F937F93B3
:103BC0008F939F93AF93BF93CF93DF93EF93FF9325
:103BD000D091E900DF708091EC00C82FC17080FDAA
:103BE000C0E81092E9008091F000877F8093F00098
:103BF00078940E940C1B1092E9008091F00088607C
:103C00008093F000CD2BCF70C093E900FF91EF912E
:103C1000DF91CF91BF91AF919F918F917F916F91E4
:103C20005F914F913F912F910F900FBE0F901F907A
:103C300018950E94F61A2FEF84E39CE021508040F3
:103C40009040E1F700C0000088E19CE00FB6F894D6
:103C5000A895809360000FBE90936000FFCF8823EB
:103C600041F08095909181038923809381030E9484
:103C70000D1A0895882339F090918103982B909321
:103C800081030E940D1A0895882321F00E94C60F17
:103C90000E940D1A0895882339F090918203982B81
:103CA000909382030E940D1A0895882391F19CEF4E
:103CB000980F913A40F4682F80EE92E00E940F072F
:103CC0000E940D1A089590E2980F983050F4877072
:103CD00091E001C0990F8A95EAF7892F0E94C60FDB
:103CE000EFCF9BE5980F933028F490E080E00E949E
:103CF0008407089598E5980F973128F490E080E0C4
:103D00000E946E070895803F20F00E94AA0C0E9436
:103D100014190895CF93C82F8823D1F18CEF8C0FFD
:103D2000813AC0F580911301882311F18091010639
:103D300087FF1EC0EC2FE695E695E695F0E0E05291
:103D4000FD4F828190E04C2F477021E030E002C0AF
:103D5000220F331F4A95E2F782239323892B89F0A0
:103D60006C2F80EE92E00E940F070E940D1A09C08E
:103D7000E2EEF2E08191C81799F382E0E83EF8079D
:103D8000C9F76C2F80EE92E00E9439070E940D1A4D
:103D9000CF91089580E28C0F883068F4C77021E0DD
:103DA00030E001C0220FCA95EAF780918203822B8E
:103DB00080938203EBCFEBE5EC0FE33040F4F0E0CF
:103DC000EE5DFE4F808190E00E948407E1CFE8E540
:103DD000EC0FE73150F4F0E0EE0FFF1FEB5DFE4F0C
:103DE000808191810E946E07D3CFC03F88F28C2FD3
:103DF0000E946F0D0E941419CBCF1F93CF93DF93B6
:103E0000182FD0E0C0E0893311F4C0E5D0E0812F55
:103E10000E948A1E209739F4812F0E94551EDF913F
:103E2000CF911F9108958FE99FE00197F1F700C0AE
:103E300000002197EFCF0F931F93CF93DF93C62FEF
:103E4000D42F022FFC0182818823A9F060933706CA
:103E50000E9408199093360680933506C77081E05A
:103E600001C0880FCA95EAF70E944B1EDF91CF91DF
:103E70001F910F91089580913706681332C0809189
:103E80003506909136060E94F918883C910548F550
:103E900010E21D0FCD17B9F080E28C0F883040F48E
:103EA000C77081E001C0880FCA95EAF70E94441EDE
:103EB000183048F481E09D2F977001C0880F9A95C3
:103EC000EAF70E944B1E802F0E94FD1E183070F6EC
:103ED000D77081E001C0880FDA95EAF70E94441E8E
:103EE000C5CFC77081E001C0880FCA95EAF7F6CF49
:103EF000B0E0A0E0EEE7FFE10C940631EC018AE0CF
:103F0000A82E2881222309F48FC02130C9F5998178
:103F10008A81913021F422960E94FD1E05C09230C4
:103F200029F422960E948A1E2196EBCF933021F429
:103F300022960E94551EF8CF943011F02196F4CFAE
:103F4000229630E020E0AE014F5F5F4F8053990B27
:103F50008A30910550F02150310930F38FE99FE00C
:103F60000197F1F700C00000F6CFA29EB001A39E1A
:103F7000700D11249C01260F371F8981EA01E3CFC0
:103F8000E22FF0E0E650FE4FB490822F86958695A2
:103F9000869590E0FC01E651FE4FE4902770F12CED
:103FA000022E02C0F594E7940A94E2F731E0E3228E
:103FB000FF24FC01E652FE4FC490D12C022E02C019
:103FC000D594C7940A94E2F731E0C322DD24FC01C2
:103FD000E653FE4F049110E002C0159507952A950F
:103FE000E2F701701127E114F10419F081EE0E944B
:103FF0008A1EC114D10419F086EE0E948A1E8B2DF0
:104000000E94FD1EC114D10419F086EE0E94551EB7
:10401000E114F10419F081EE0E94551E01151105FD
:1040200009F482CF8CE278CFCDB7DEB7EAE00C940A
:1040300022319091020692FF10C098E0899F900172
:104040001124622B609360030E94E51A0E940819F4
:1040500090935F0380935E0308950E94E51A08958C
:10406000A7E1B0E0E6E3F0E20C940D314B8B5C8B02
:104070006D8B7E8B8F8B6111109281031A8A198A46
:1040800085E0FE017396DE011D9601900D928A95E2
:10409000E1F78091020682FF1CC00E94081920915E
:1040A0005E0330915F03821B930B8838934120F0AD
:1040B0008091600382FF78C00E94081920918303D9
:1040C00030918403821B930B8838934110F00E9437
:1040D000BB0F86E0FE013D96DE01179601900D9222
:1040E0008A95E1F7CE0107960E94A627811112C09A
:1040F00086E0FE013796DE01119601900D928A95B9
:10410000E1F78A859B85892B29F088859F81892302
:104110008F3F81F516E080915D0390912C03891308
:1041200017C06796E3E00C94293196E0929FD00186
:10413000939FB00D1124A35DBC4FFE0131960190F9
:104140000D929A95E1F780932C030E94D40FE2CF51
:10415000819FC0011124835D9C4F0E94A627882364
:1041600001F380915D0390E0019687709927809319
:104170005D03D1CF20912C0330E0C90101968770F7
:10418000992740915D034817190679F60E94F61A9F
:1041900010922C0310925D0386E0E6E2F3E0DF016B
:1041A0001D928A95E9F7B6CF82E00E94AD1A84CFBE
:1041B000A5E0B0E0EEEDF0E20C940C318C019093B0
:1041C000F3058093F205011580E21807C0F4802FF3
:1041D0000E94551EC8010E9449109801205E3109B5
:1041E0002830310518F00115110531F40E94441EE4
:1041F0002596E4E00C9428310E942F1EF9CF80EF21
:1042000089838A831B820E9408198160782F9D838D
:104210008C8349815A816B818D810E943020E8CF47
:10422000A5E0B0E0E6E1F1E20C940C318C01909352
:10423000F3058093F205011580E21807C0F4C80168
:104240000E9449109801205E31092830310518F08C
:104250000115110549F40E944B1E802F0E948A1EF1
:104260002596E4E00C9428310E943A1EF6CF80EFA8
:1042700089838A8381E08B830E9408198160782F6B
:104280009D838C8349815A816B818D810E9430206E
:10429000E7CFA5E0B0E0EFE4F1E20C9404316C016B
:1042A000FC0183819481892B31F080819181892364
:1042B0008F3F09F058C52596ECE00C9420310E9400
:1042C0002812182F682F89819A810E941210698103
:1042D0007A81812F0E940B128C01F6018281882342
:1042E00009F436C5980122513F452031310508F0C7
:1042F00008C58FEF93E00E9404328111A5C00251DE
:1043000057EFA52E52E0B52E011133C019821A8243
:104310001B821C82EE24EA9445013FEF831A930A24
:10432000C5010E94043289831A82882309F48CC053
:10433000813009F07EC085010E5F1F4FC4010E94CD
:104340000432F82E8A83882309F47EC0C8010E94B3
:104350000432982E8FEF8F0D8330D0F40F5F1F4FF4
:104360009B82992021F0CE0101960E94781F58016E
:10437000D3CFA114F4E0BF0609F466C0C5010E94C2
:104380000432811101C001502FEFA21AB20ABCCF32
:104390008BEF8F0D833040F5C50103969B828C0116
:1043A000992029F385010C5F1F4F0E9404328C83F2
:1043B0008823E9F2AB80BC8041E0A4164FEFB4063D
:1043C00010F0BA2CAA2456E0F51651F087E0F81642
:1043D00019F0C5010E941021C5010E94D820C7CF45
:1043E000C5010E941021C3CF94E0F912C0CF85010E
:1043F0000C5F1F4FC50103960E940432992021F1E2
:10440000882311F18150990BE89E9001E99E300DAF
:104410001124E92DE150FF0BCF01820F931F01976B
:1044200008F4A5CFEFE9FFE03197F1F700C00000F5
:10443000F6CFCE0101960E94781F840198CF81E0CB
:104440000E94E51A0E94941A80916003877009F413
:1044500032CFF6018281882309F42DCF80910206A4
:1044600082FF29CF82E00E94AD1A25CF81E00E9411
:10447000A01AE8CF82E0E4CF053FECE51E0709F47F
:1044800061C008F45BC0063F2CE5120709F45EC06A
:10449000882309F479C41092370603303DE51307E9
:1044A00008F05BC00A3F4CE5140730F4C8018250A5
:1044B0009C45449708F05BC00E949D1290930206B1
:1044C0008093010601319CE5190709F42DC108F01C
:1044D000A7C00930FCE51F0709F414C108F072C039
:1044E00005303CE5130709F405C108F057C0033057
:1044F0005CE5150709F4F4C008F0F8C080910106E6
:10450000816002309CE5190709F4EDC06091010655
:104510001091020684E090E00E942232612F82E234
:1045200090E00E9422320E94F61A8ECF27E245EEDA
:1045300065EE0AC426E241EE60EE06C427E245EECF
:1045400064EE02C426E241EE62EEFEC327E245EECF
:1045500066EEFAC328E241E0EBCF01365DE51507D0
:1045600009F4AACF053A8DE5180709F4A5CF06315D
:10457000ECE51E0709F077C4809182038A7A91E006
:1045800009F490E09093000369E2811165E380EE05
:1045900092E00E9439070E940D1A56CF80910106C1
:1045A00080620730ECE51E0709F49DC0809101068A
:1045B00080610830FCE51F0708F495C08091010672
:1045C000806491C0809101068B7F0D302CE512072D
:1045D00009F489C0A0F4809101068E7F0B304CE570
:1045E000140709F480C0809101068C600C305CE5F2
:1045F000150708F478C0809101068D7F74C00F30D4
:104600008CE5180709F48CC080910106877F003182
:104610009CE5190708F467C0809101068F7D63C08F
:104620000D3FECE51E0709F477C058F505312CE580
:10463000120709F483C098F480910106837F033147
:104640004CE5140709F44FC008F472C00E94F61A32
:1046500090910106892F97FB87F9805844C00B3F42
:104660008CE5180709F44AC008F052C08091020690
:1046700081600A3FECE51E0709F048CF80930206EF
:1046800045CF0130FDE51F0709F464C0C0F48091F7
:1046900002068C7F0F3F3CE5130781F380910206F1
:1046A000836001154DE5140748F380910206982FA9
:1046B000909591708E7F892B90FB81F9DFCF013629
:1046C0005DE5150709F44CC0053A8DE5180709F4B6
:1046D0004EC002309DE5190709F018CF60E03BC0DD
:1046E0008091010682608093010610CF80910106BF
:1046F0008460F9CF809101068860F5CF8091020631
:104700008260BCCF0E94F61A809101068068EBCFD0
:10471000809102068E7FB2CF809102068D7FAECF50
:10472000809101068F7EDFCF809101068F7BDBCFEA
:104730000E94F61A809101068F77D5CF80910106ED
:1047400082FB992790F921E0922790FB82F990FB58
:1047500083F9C9CF61E08EE090E00E942232D6CE8C
:1047600090910106892F8F7E94FF8061BCCF90913C
:104770000106892F8E7F90FF8160B5CF8091000365
:1047800069E2811165E380EE92E00E940F0703CF9A
:1047900043E458E06EE478E00E94A70755CE4EE46B
:1047A00058E063E478E0F8CF44E158E06FE178E066
:1047B000F3CF4FE158E064E178E0EECF48EF57E007
:1047C00066E078E0E9CF46E058E068EF77E0E4CFD4
:1047D0004AEE57E06CED77E0DFCF4DEA57E06BEB48
:1047E00077E0DACF4BEB57E06DEA77E0D5CF61E0C9
:1047F00081E00E942A0828CE61E085E0FACF0E947D
:10480000F61AFFEF24E33CE0F15020403040E1F79E
:1048100000C000000E940F118091020682FB8827D1
:1048200080F991E089270E94C91AF60182810081EE
:104830001181882309F445C0C8010E942812F82E6E
:10484000682FC8010E941210B8018F2D0E940B1210
:104850000E94330E8C01882EF601E280B580B2945E
:104860003FE0B322809160038770C1F0AE2CEE2050
:10487000B1F0812F807F803421F080E2800F88307A
:1048800068F08091020682FF09C082E00E94AD1AA2
:10489000809160038770AA24A3948111A12C912E8A
:1048A00092942FE09222FBE0F91508F476C0E92DEE
:1048B000F0E0E953FD4C0C94493181E0B4CF80E045
:1048C000B2CFC8010E94DE0FF82EBECF212F2F706D
:1048D000F22E107F19F0F29490EFF922EE20B9F049
:1048E000FF2069F080E2800F883010F0811009C04D
:1048F00080918203F82AF09282030E940D1A802F81
:104900004AC080918103F82AF0928103F6CF802F6C
:104910000E94551EFF2009F440C0005E083010F0D0
:10492000811004C08F2D0E94C60F06C0F0948091A4
:104930008103F822F09281030E940D1A2EC0312FBC
:104940003F70F32E107F103219F0F29480EFF822AE
:10495000882089F041E0841609F491C0EE2009F422
:104960009AC0BB2009F467C0F601858180FFC7CFDC
:104970008F70858360C08091020682FD35C0EE2075
:1049800069F1FF2039F080918203F82AF0928203C6
:104990000E940D1A80E00E948A1E292D2850330B98
:1049A0002430310510F40E949A07AA2009F483CC20
:1049B0008091600380FD7FCCF601128285958595FC
:1049C00085950E94E51AC6010E94492180916003E5
:1049D0008595859585950E94A01A6DCC80E00E94F2
:1049E000551EFF20D1F29ECFEE2049F1B11004C038
:1049F000809185038F2920C051E0B51210C082FF3D
:104A0000CCCF80918503F82AF81639F20E94081954
:104A10009093840380938303F0928503BECF85E057
:104A2000B812E6CF0E94BB0F909101038F2D892B06
:104A30008913809301038F2D0E944B1EAECFB110BE
:104A400003C00E94BB0F12C091E0B91213C0809145
:104A500082038F2109F4A1CF0E94BB0F9091010323
:104A60008F2D809589238913809301038F2D0E94B8
:104A7000441E93CFE5E0BE1609F48FCFE2CFEE20BF
:104A800029F0F5E0FB1508F488CFD5CF24E02B15ED
:104A900008F483CFEBCFBB2049F3F9E38F1209C0B1
:104AA0002FEF37EE43E0215030404040E1F700C0A7
:104AB0000000802F0E94551E70CF812F869586950D
:104AC000837061F0813009F068CFC8019370E11004
:104AD00002C090E080E00E946E075FCFC801937033
:104AE000E11002C090E080E00E94840756CF802F42
:104AF000EE2029F00E946F0D0E9414194ECF0E94E3
:104B0000AA0CFACF812F837089F5E11046CF402F90
:104B1000429546954770440F440F802F8F70042EA6
:104B200001C0880F0A94EAF7202F207104FF07C004
:104B30002FE030E001C0220F4A95EAF72095169544
:104B400016951370123069F050F4309186031130CD
:104B500029F0822B83230E94F11A1FCF832B822BF3
:104B6000FACF282B809186038227F5CF8695EE20F9
:104B700011F0812F8170882309F40FCF402F4295C7
:104B800046954770440F440F802F8F70042E01C04C
:104B9000880F0A94EAF7202F207104FF07C02FE046
:104BA00030E001C0220F4A95EAF720951695169538
:104BB0001370123069F050F430913806113029F03A
:104BC000822B83230E948F1AE8CE832B822BFACF6D
:104BD000282B809138068227F5CF1F70EE2029F010
:104BE000812F0E94E51A802F27CF802F0E94441E1C
:104BF000812F0E94A01AD1CE802F52EF8516B1F1DD
:104C0000581570F090EF8916D1F0E1EF8E1691F003
:104C1000EE2009F466C0B11072CE812F8F712AC0C8
:104C2000F3EF8F1651F124EF8212F2CF809102063A
:104C300082FD2FC0812F8F71EE20D9F21BC0EE2094
:104C400081F034E03B1508F4A8CE1F7181E090E0BC
:104C5000012E01C0880F0A94EAF79091380689273F
:104C6000B1CF45E04B1508F498CEEFCF812F8F716F
:104C7000E110BFCF0E94E51A90CE80E0EE2009F44B
:104C8000A1CF1F7181E0012E01C0880F0A94EAF7BD
:104C900099CFEE20C9F0809160038770843041F491
:104CA0000E94CD0F812F8F710E94A01AA12C75CE6A
:104CB00054E05B15D8F31F71812F0E94E51A63E061
:104CC000812F0E941920F2CF84E08B1530F40E94CE
:104CD000CD0F64E0812F8F71F4CF81E00E94AD1A77
:104CE000E5CFBB2059F0893309F0E3CE9FEFE7EE23
:104CF000F3E09150E040F040E1F7D9CE812F8F7181
:104D000078CF0031FFE51F0709F499CB01312FE57A
:104D1000120709F4AFCB033F2CE5120709F40ACCC4
:104D200008F0AACB083D4CE5140709F4FFCB093D78
:104D30005CE5150709F40ECC073D9CE5190709F061
:104D4000A7CB26E241EE61EEC6010E941B1F7CCB81
:104D500000313FE5130709F489CB01314FE5140712
:104D6000D1F682E084CB85E0DE01119601900D92B0
:104D70008A95E1F7F601228189819A8121119FCAE2
:104D80000E94DE0F182FA3CA0631FCE51F0709F4A5
:104D9000F5CC8091820382720A3C2CE5120709F45B
:104DA00017CDB0F5053C4CE5140709F4FDCCD0F463
:104DB000033C9CE5190709F4EBCC08F0F0CC023C6D
:104DC000FCE51F0709F031CD80913D0691E0892770
:104DD00080933D06109212018091EF0381608093D1
:104DE000EF0332CB073C2CE5120709F4E7CC08F4BB
:104DF000E0CC083C4CE5140709F4E5CC093C5CE543
:104E0000150709F012CD4CED57E06AEE77E0C4CCFF
:104E10000F3C9CE5190709F4EFCCA0F40C3CFCE531
:104E20001F0709F4DFCC08F4D8CC0D3C3CE5130790
:104E300009F4DDCC61E082E00E3C4CE5140709F496
:104E4000D8CCF3CC063D5CE5150740F4013D8CE57C
:104E5000180708F0F9CA61E088E0CBCC0D351007DF
:104E600009F4F2CAE2CC0A35EDE51E0709F425CDB6
:104E700068F401152CE5120709F4C1CC0E3D1C4560
:104E800009F0D3CC0E9491170E94191E0C354DE5F4
:104E9000140709F4C1CC08F412CD073A1D45A1F35B
:104EA000C4CC1F93CF93DF9380912B03807F09F0B5
:104EB00049C080912803882309F444C080915D0390
:104EC000D0912C036091260370912703A0912903B0
:104ED000B0912A03C62FC72316E0D81799F190E0A6
:104EE000109711F0CF3F19F401968770F6CF189FF5
:104EF0009001199F300D1124F901E35DFC4F4181B0
:104F00004713F2CF40814613EFCF42814111ECCFDE
:104F1000438154814A1B5B0B483C510528F7809123
:104F20002B038F70806180932B03F901EE5CFC4FA3
:104F300080818F708061808386E293E00E944921A6
:104F40000E94D40FDF91CF911F910895A1E1B0E0AD
:104F5000ECEAF7E20C9406318C0185E0F801DE0101
:104F60001D9601900D928A95E1F7F801E28086E2A4
:104F7000A82E83E0B82E6091290370912A03611551
:104F8000710509F426C19091260340912703892FCA
:104F900084238F3F09F41DC120813181C380D480D7
:104FA000F0902803F601E61BF70BFF2009F4DCC0A4
:104FB00080912B03582F507FE83CF10508F09FC0EB
:104FC00051116BC0FE2C431314C0921312C0E11098
:104FD00010C08F70806180932B03C5010E9449210E
:104FE00080912B03F80185838F2D6196EAE00C9464
:104FF0002231C114D10429F0822F83238F3F09F07D
:1050000003C180E0F82FF170DF2E80FF3CC080915B
:105010005D0340912C0356E0841315C02D873E8715
:105020008D859E850E945712292F22952F70223040
:10503000F0F0243018F59F70F1F0F8019581907F21
:10504000D1F4D12C1EC090E0589FF001599FF00D73
:105050001124E35DFC4F6181361306C06081261385
:1050600003C06281E6120FC001968770D5CF9F7092
:1050700011F0882331F3805E883018F3C8010E9454
:105080004921FD2CB1CFEE2009F4AECF80912B0346
:10509000816080932B03F12CA7CF431306C092139A
:1050A00004C0F801EE2009F479C0C8010E9464121E
:1050B000882309F1EE20F9F080912B03803270F003
:1050C000209126033091270338872F831986DB86AA
:1050D000CA868C87CE0107960E94492186E0F80196
:1050E000A6E2B3E001900D928A95E1F70E94512764
:1050F000FF24F39479CFC8010E944921F9CF5111BF
:105100000AC086E293E00E94492186E0F5011192EF
:105110008A95E9F7C0CF43130FC092130DC0E11079
:105120000BC0F8018583C8010E94492186E0F50182
:1051300011928A95E9F758CFC8010E94641288231A
:10514000D1F2EE20C1F280912B03803238F220910F
:105150002603309127033A8329831B82DD82CC8288
:105160008E83CE010196B8CFE83CF105F8F6FE2C0F
:10517000EE2009F243131FC092131DC080912B0330
:1051800080FD10C0982F907F69F0F8018583903FD3
:1051900031F0982F907F905F8F70892B8583C801A5
:1051A0000E94492186E0F801A6E2B3E001900D9249
:1051B0008A95E1F719CFC8010E94641281118ECF40
:1051C00080912B03816080932B03C8010E944921A9
:1051D0000BCFEE2009F48FCFC8010E946412F82E85
:1051E000882309F488CF86E0F801A6E2B3E00190B5
:1051F0000D928A95E1F780912603909127030E94F2
:1052000057120E945127F0CE81E08E25FBCE1F92CF
:105210001FB61F9211248F939F93AF93BF938091DA
:10522000FC05811113C08091FD059091FE05A091B0
:10523000FF05B09100064196A11DB11D8093FD05AB
:105240009093FE05A093FF05B0930006BF91AF9128
:105250009F918F911F901FBE1F901895CDB7DEB7FD
:10526000E4970FB6F894DEBF0FBECDBF85B7806858
:1052700085BF85B7806885BF84B7877F84BF0FB639
:10528000F894A895809160008861809360001092E6
:1052900060000FBE80E890E00FB6F8948093610044
:1052A000909361000FBE87ED9DE09093DF028093A5
:1052B000DE020E945F050E9452068091E200846037
:1052C0008093E2007894809134068823A1F01091B5
:1052D000E9001F709091EC00892F817090FD80E8AB
:1052E000182B1092E9008091E80083FD0E940C1BAE
:1052F0001F701093E90082E084BD93E095BD9AEFA2
:1053000097BD80936E000E948412811102C00E949A
:10531000CC1103E511E029E5E22E21E0F22ED801BF
:105320008D918D018F3F11F00E94D90DE016F1068D
:10533000B1F709E511E0F80181918F018F3F11F07C
:105340000E94D90DF1E008361F07A9F78CE0E8EAC2
:10535000F3E0DF01282F1D922A95E9F7EAE8F3E050
:10536000DF011D928A95E9F70E948517811102C01D
:105370000E94911782E090E00E940432809396038D
:105380000E949D1290930206809301060E943B1991
:10539000EFEBFDE53197F1F700C000000E943B19EB
:1053A0008091A80380FF08C06FEF7FEF90E080E05E
:1053B0000E9440320E940F1183E090E00E9404326C
:1053C0000E94F11A0E94CC13109243068FEF9FEFB8
:1053D00090935D0680935C0690935F0680935E06D3
:1053E00090936106809360069093630680936206B3
:1053F0009093650680936406909367068093660693
:10540000909369068093680690936B0680936A0672
:105410001092C1039093DB038093DA039093DD0332
:105420008093DC039093DF038093DE039093E1038A
:105430008093E0039093E3038093E2039093E5036A
:105440008093E4039093E7038093E6039093E9034A
:105450008093E8030E948517811104C00E94911770
:105460000E94711746E050E06CE170E08DE396E039
:105470000E94F4311092EF0380913D068C7F11F46D
:105480000E94711784E091E09093F9058093F805EC
:10549000332433948091340600E112E1853009F41D
:1054A000F9C00E943B19882359F08FB7F8944091B6
:1054B000FD055091FE056091FF05709100068FBFBC
:1054C00098EAE92E93E0F92EE7E9F3E0D70110E03E
:1054D00000E0602FCD90DD90219131912C153D059C
:1054E00009F420C2912CAA24A394B12C2C253D258B
:1054F000A9014A215B21452B09F40EC299A66AA78E
:10550000CA20DB2081E0C114D10409F480E08BA71C
:105510000E9408198160782F9DA78CA749A55AA5DC
:105520006BA58DA50E943020F801EE0FFF1FE956F4
:10553000FC4F80819181A826B926B182A082CD2816
:1055400071F08FE0809FF001819FF00D1124E158F0
:10555000FE4FE90DF11D80818F3F09F0A7C0B12CEE
:105560000B2D10E08091C103800F912F911D0997A1
:105570006CF188E090E06C01C01AD10AB8016E535A
:105580007C4FA60182EC93E00E94E431B80166539F
:105590007C4FA6018AEC93E00E94E431A601440FFF
:1055A000551FB801660F771F66527C4F8AED93E056
:1055B0000E94E431B8016E527C4FA60182ED93E067
:1055C0000E94E43188E08B198093C1038091C1036C
:1055D00090E0A22DB0E09D01220F331F27523E4FD5
:1055E000AA0FBB1FBD0166527E4F78C08091340662
:1055F000843009F43EC08091EE03811105C00E9401
:10560000B01480E00E945A08F1E0F093EE030E948B
:10561000A1168091EE03811105C00E94B01480E0B4
:105620000E945A0821E02093EE031092FC0588E1C5
:1056300090E0A0E40FB6F894A895809360000FBEA8
:10564000A093600083B7817F846083BF83B781604C
:1056500083BF7894889583B78E7F83BF0FB6F89405
:10566000A89580916000886180936000109260002E
:105670000FBE80912A06882369F00E943B19E8EA50
:10568000F3E081919191892B09F0B8C4B3E0E43B38
:10569000FB07B9F780913406853009F4A7CF0E9443
:1056A000F61A0E949A071092EE03FBCE282EBB2416
:1056B000B39456CF90E0FC01EF53FC4FD9015C91BD
:1056C0005183DB015C915187218A880F991FFC016E
:1056D000EF53FC4F128E118E91E0842F41E0480F62
:1056E0009B1540F38093C1030E94A11686E0EBEB6B
:1056F000F3E08E010F5F1F4FD80101900D928A9544
:10570000E1F71092BD031092BE031092BF031092F6
:10571000C0038B819C81892B09F44AC08091B90315
:105720009091BA030E94F9189C019091B5039923B6
:1057300009F487C425313105D8F19F3F19F09F5FE7
:105740009093B503DB80DD2059F00E944F0D9FEF51
:105750001D140CF491E0899F802D11248093BD03CA
:10576000DC80DD2059F00E944F0D9FEF1D140CF4DA
:1057700091E0899F802D11248093BE033091BD0359
:105780003323B1F02091BE03222391F045EB340383
:10579000C0011124992309F4DCC09093BD0345EBAB
:1057A000240390011124332309F4D6C03093BE039F
:1057B0008D819E81892B09F44AC08091B703909115
:1057C000B8030E94F9189C019091B403992309F43D
:1057D00033C421353105D8F19F3F19F09F5F909375
:1057E000B403DD80DD2059F00E942D0D9FEF1D14C4
:1057F0000CF491E0899F802D11248093BF03DE80FB
:10580000DD2059F00E942D0D9FEF1D140CF491E046
:10581000899F802D11248093C0033091BF033323CF
:10582000B1F02091C003222391F045EB3403C00175
:105830001124992309F493C09093BF0345EB2403EB
:1058400090011124332309F48DC03093C00346E046
:1058500050E0B8018BEB93E00E94D731892B61F4C3
:105860008091BD039091BE03892B9091BF03892B3A
:105870009091C003892B11F00E94141986E0F80161
:10588000ABEBB3E001900D928A95E1F70E949A0785
:105890009091A30389138093A303809134068430ED
:1058A00009F0F8CD83E08093E9008091E80082FF61
:1058B000F1CD8091E80090E085FF0AC00E947E054E
:1058C00030E2A32EB12C6801882309F458C091E07E
:1058D0008091E8008B778093E800992309F4DACD72
:1058E000C090F405D090F5058981C114D10409F464
:1058F00054C08E3F09F0E5C08A81833020F0855086
:10590000833008F0DEC0EA81EE3008F0DAC0F0E063
:10591000ED52FD4C0C9449319394AA0CBB1C4FE002
:105920009412E6CD0F5F1F4F0630110509F0D1CD5F
:105930008FEF8EA78FA718AA0E9408198160782F71
:105940009AAB89AB4EA55FA568A98AA90E943020B1
:10595000CBCE3092BD0323CF3092BE0329CF3092FD
:10596000BF036CCF3092C00372CF8091F100D6019B
:105970008D936D01B1E0AB1AB10809F4A8CF809105
:10598000E80085FDF2CF8091E8008B778093E800F6
:105990000E947E05882399F39ACF8B3009F440C288
:1059A00058F5853009F4B7C0D0F4823009F46FC0DF
:1059B00030F4813009F467C08FEF898382C083306F
:1059C00009F49AC08430C1F74C816B818A810E94AE
:1059D000DC119827892798279E838D8372C0873092
:1059E00009F4A7C008F4A2C0883009F4DFC08930E8
:1059F00019F70E94961665C0803109F462C1B8F5A6
:105A00008D3009F432C108F42DC18E3009F42FC154
:105A10008F3091F68091F0059091F105892B09F472
:105A200050C0EC80F12CFDE1EF16F10408F049C004
:105A3000CA80DB80DC24CD24DC245801E00EF11E7A
:105A4000C60189509D4FAE14BF04D9F129E0C2169A
:105A500021E0D20628F4D50114966C910E942232DE
:105A6000BFEFAB1ABB0AEFEFCE1ADE0AE9CF8231E5
:105A700009F42CC108F428C1833109F450C18E3FC8
:105A800009F09ACF40CF1A8289E08B831AC08A81AD
:105A9000823009F4C9C28330C1F0813009F08CCF63
:105AA0002FB7F8946091FD057091FE058091FF0578
:105AB000909100062FBF0E944F316B837C838D83B2
:105AC0009E83C8010E94D905E5CC8091F005909194
:105AD000F105892BB1F3F801D7018C9111969C91B6
:105AE000B2E0EB0EF11C92838383329624EBE21634
:105AF00023E0F20689F7E5CF8A81823009F05CCF96
:105B00006B817C818D819E810E944F3186E290E085
:105B10000E942232D6CF2D813E8132272327322781
:105B20004C816B818A810E944311CBCF0E94691105
:105B3000C8CF8A81813429F64B815C8180913D06F2
:105B4000982F93704115510589F49111109212010B
:105B50008C7F80933D068D81809341068E8120E06D
:105B600048856F8190E00E94C907ABCF911102C0B8
:105B7000109212018C7F816080933D0626E234E012
:105B80006EE674E0F901329685919491F901A59140
:105B9000B4914A175B0731F02C5F3F4F62177307D0
:105BA00089F780E060E00E942A08D5CF8A8181349D
:105BB00059F0823409F436C0803409F082CF3B8238
:105BC0001C8288EC8D837DCF80913D06982F937049
:105BD000C1F08695869590E026E234E06EE674E0AA
:105BE000F9013296A591B491F90145915491E42FB0
:105BF000452F8A179B0739F02C5F3F4F62177307B9
:105C000079F7E0E040E0EB834C83809141068D839F
:105C100080913E068E8380913F068F83809140065F
:105C200088874FCFEB80FC804EE150E06FEF70E053
:105C3000CE0103960E94ED3186E294E0DE011396D8
:105C40002EE1FC0145915491E416F50628F422302A
:105C500018F04D935D932250049634E08E369307EE
:105C600081F72FCF80E18A832CCF3A820DCFEC8051
:105C7000F12C4DE1E416F10408F023CFCA80DB805B
:105C8000DC24CD24DC245801E00EF11EC60189502D
:105C90009D4FEA14FB0409F414CFA9E0CA16A1E051
:105CA000DA0658F40E940432F5018483BFEFCB1A60
:105CB000DB0AEFEFAE1ABE0AE9CFD50114961C92AB
:105CC000F5CF0E943311FDCE84E0CDCFEC80F12CD6
:105CD000FDE1EF16F10408F0F4CECA80DB80DC248D
:105CE000CD24DC245801E00EF11EC6018796EA148B
:105CF000FB0409F4E6CE20EDC21622E0D20660F4E1
:105D00000E940432D50114968C93FFEFCF1ADF0A5C
:105D10002FEFA21AB20AE9CFF5011482F6CFCC8098
:105D2000D12C3DE1C316D10408F0CBCEEA80FB8034
:105D3000FE24EF24FE2440EDE41642E0F40608F0D1
:105D4000C0CE80ED92E08E199F098C159D0508F458
:105D5000B8CE370187E2680E711C8091F0059091F2
:105D6000F10527014C0C5D1C892BB9F5570191E019
:105D7000A922BB24E0FE0DC0C70186960E94043212
:105D80009D8189279827892781159C4511F48FEFDC
:105D90008D83460140FE1AC0B1E08B1A9108E5E000
:105DA000F0E0EC0FFD1FE80DF91DFCABEBABC30100
:105DB0008C0D9D1D0E940432ABA9BCA99C9181153C
:105DC0009C4521F48FEFEBA9FCA98083F801EA0D33
:105DD000FB1D2FEFA814B90410F068011BC09481BB
:105DE000858181159C4511F42483258342E0A40E0E
:105DF000B11C3296EFCFA0EDEA16A2E0FA0620F42D
:105E0000F60164810E942232FFEFCF1ADF0A2FEFE2
:105E1000E21AF20AC70187964E145F0461F751CE69
:105E20008091F0059091F105892B09F44ACEC801C3
:105E30000E94D9053FEF41EE84E031504040804060
:105E4000E1F700C00000B6CA88E0EAE1F1E0DE0157
:105E5000919601900D928A95E1F780E2D8011D920A
:105E60008A95E9F785E0898388E0FE01B196DE0135
:105E7000159601900D928A95E1F73D8622CE8CEA27
:105E800089833A821B821C821CCE8C81682F70E031
:105E9000762F66278B81860F972F911D092E000C78
:105EA000AA0BBB0B25E0880F991FAA1FBB1F2A95C1
:105EB000D1F7AC01BD01405E5F4F6F4F7F4F481778
:105EC00059076A077B0708F4FCCD8C3AE1E09E078E
:105ED000A105B10508F0F5CD4D3AF1E05F07610588
:105EE000710520F04CEA51E060E070E0481B590B6E
:105EF000BC0166587D4FC8010E94CE31E2CD4AE117
:105F000050E06FEF70E0CE0107960E94ED31809176
:105F1000F0058983CA821B821C8283E08D838DE019
:105F20008E83CFCD81E090E09093F5058093F405CA
:105F300082E390E09093A7038093A6030E94081940
:105F40009093A5038093A403BCCDCD2889F1D09074
:105F5000A803E090AE03F090AF038091A40390916A
:105F6000A5030E94F9188536910558F1F5FAEE243B
:105F7000E0F8EE2031F1D0FE24C00E940819909381
:105F8000A5038093A4038091A6039091A703019792
:105F90009093A7038093A603892B51F41092F505E3
:105FA0001092F40581E090E09093F1058093F00564
:105FB0008091F00589838091F4058A838091A603FE
:105FC00064CD82E390E09093A7038093A603F0CF83
:105FD0001092F1051092F00574CD40E250E06FEFA1
:105FE00070E0C8010E94ED316CCD8B81811169CDCB
:105FF00080E2D8011D928A95E9F763CD09BD19BDEC
:1060000009B400FEFDCF8091D8008F7D8093D80029
:106010008091E00082608093E0008091E00081FD4B
:10602000FCCF0E94F61A36CB86E290E00E94043242
:106030001B821C821D8274CF2B30310508F0CECB21
:1060400006CC2B30310508F07ACBB2CB1092B900D8
:106050008CE08093B8000895B0E0A0E0E2E3F0E3C4
:106060000C940531B82EEB010E9408196C01EE2446
:10607000E394F12CC431D10560F025E0E22EF12C3F
:10608000CF3FDC0731F0CE0164E170E00E94EA30DE
:106090007B0184EAA82E94E8992E1092BC00A0926D
:1060A000BC000E9408198C018091BC0087FF0DC0C4
:1060B0008091B900887F883001F18091B900887F94
:1060C0008031D9F00FEF1FEF09C00E940819801B23
:1060D000910B8E159F0540F30EEF1FEFCF3FDC07AE
:1060E000E1F2C6010E94F9188C179D07B0F2C801B1
:1060F000CDB7DEB7EBE00C942131B092BB009092AB
:10610000BC000E9408198C018091BC0087FF0AC066
:106110008091B900887F883111F0803499F610E0C1
:1061200000E0E5CF0E940819801B910B8E159F059A
:1061300058F3D2CF0F931F93CF93DF93EB0180934C
:10614000BB0084E88093BC000E9408198C018091F8
:10615000BC0087FF11C02091B900287F81E090E04A
:10616000283211F490E080E0919581959109DF91BA
:10617000CF911F910F910895CF3FDC0741F30E940B
:106180000819801B910B8C179D0708F38EEF9FEF6A
:10619000EECFB0E0A0E0EFECF0E30C9408316B013F
:1061A0008A017901B9010E942C30E6010C0D1D1DF8
:1061B000C017D10711F097FF08C024E92093BC0055
:1061C000CDB7DEB7E8E00C942431B70189910E9485
:1061D0009A30EECFAA1BBB1B51E107C0AA1FBB1F01
:1061E000A617B70710F0A61BB70B881F991F5A9563
:1061F000A9F780959095BC01CD0108952F923F920B
:106200004F925F926F927F928F929F92AF92BF92C6
:10621000CF92DF92EF92FF920F931F93CF93DF9372
:10622000CDB7DEB7CA1BDB0B0FB6F894DEBF0FBECF
:10623000CDBF09942A88398848885F846E847D841C
:106240008C849B84AA84B984C884DF80EE80FD801E
:106250000C811B81AA81B981CE0FD11D0FB6F89494
:10626000DEBF0FBECDBFED01089597FB072E16F4DC
:10627000009407D077FD09D00E94EA3007FC05D0D2
:106280003EF4909581959F4F0895709561957F4F4D
:106290000895EE0FFF1F0590F491E02D09946927F2
:1062A000962769277827872778270895CF92DF9246
:1062B000EF92FF92CF93DF93CDB7DEB72A970FB659
:1062C000F894DEBF0FBECDBF89879A87A985BA85AE
:1062D0002D913D914D915C9129833A834B835C8351
:1062E000232B242B252B41F424E239ED4BE557E0F9
:1062F00029833A834B835C8369817A818B819C817A
:106300002DE133EF41E050E00E94463269017A010D
:10631000A7EAB1E49B01AC010E94653269837A83EC
:106320008B839C83ACEEB4EFA70196010E9473327D
:106330009B01AC0189819A81AB81BC81820F931F43
:10634000A41FB51FB7FF03C00197A109B048E98595
:10635000FA8580839183A283B3839F772A960FB6B1
:10636000F894DEBF0FBECDBFDF91CF91FF90EF90CD
:10637000DF90CF9008950E945631089580E091E01B
:106380000E9456310895B0E0A0E080930001909300
:106390000101A0930201B09303010895FB01DC0108
:1063A00002C005900D9241505040D8F70895FB016E
:1063B000DC0104C08D910190801921F441505040BE
:1063C000C8F7881B990B0895FB01DC0102C00190FE
:1063D0000D9241505040D8F70895DC0101C06D93F3
:1063E00041505040E0F70895DC01CB01FC01F999E0
:1063F000FECF06C0F2BDE1BDF89A319600B40D9211
:1064000041505040B8F70895F999FECF92BD81BD33
:10641000F89A992780B50895A8E1B0E042E050E0ED
:106420000C94F631DC01A40FB51F4150504048F0E8
:10643000CB01840F951F2E910E9423324150504072
:10644000D0F70895262FF999FECF92BD81BDF89A15
:10645000019700B4021639F01FBA20BD0FB6F894A8
:10646000FA9AF99A0FBE08950396272F0E942332B5
:106470000E942232252F0E942332242F0C94233293
:106480000196272F0E9423320C942232052E97FB6F
:106490001EF400940E945D3257FD07D00E947832AE
:1064A00007FC03D04EF40C945D3250954095309526
:1064B00021953F4F4F4F5F4F089590958095709570
:1064C00061957F4F8F4F9F4F08950E949A32A59FED
:1064D000900DB49F900DA49F800D911D11240895DF
:1064E000B7FF0C9465320E946532821B930B0895AE
:1064F000A1E21A2EAA1BBB1BFD010DC0AA1FBB1FC8
:10650000EE1FFF1FA217B307E407F50720F0A21B39
:10651000B30BE40BF50B661F771F881F991F1A94A6
:1065200069F760957095809590959B01AC01BD01D0
:10653000CF010895A29FB001B39FC001A39F700D2A
:10654000811D1124911DB29F700D811D1124911D7B
:106550000895F894FFCFE014EC141C15611566152E
:106560006C156F1572157515DA15DD152B16671676
:106570006C166F167C1687169216ED1B151CC31D24
:10658000151CC31D481C691CC31D721D7F1D66247C
:1065900066249F249F245D257725CD24CD24822544
:1065A000ED25FC25FC25242F3F2F452F612D612D46
:1065B0007F2F922FA52FE82FED2F612D612D612DBB
:0265C000F52FB5
:1065C200010000000C07CF10AE10A910A4100B0799
:1065D200FFFF030100FF0000FFC87E49EB6FA42606
:1065E200441C818283E200E900EA00B500B600B7EC
:1065F20000CD008301CC008A019201940121022383
:106602000224022502260227022A02B300B4006FE6
:10661200007000F7F6F5F4F1F0303132333792932F
:106622009594969734353666003131295A1B750A8E
:106632004022BC8A016801AC00AC09C509E5090029
:106642000102030405060708090A0B0C0D0E0F10C0
:106652001112131415161718191A1B1C1D1E1F20B0
:106662002122232425262728292A2B2C2D2E2F30A0
:106672003132333435363738393A3B3C3D3E3F4090
:10668200414243444546474849FF4A4B4CFF4D4E21
:106692004F50FF515253545556000010001E002B0C
:1066A200003800480055006300700080008D009A99
:1066B20000A700BE00D800000D100D200C310E42C4
:1066C2001052145C1A66147610860E960CA70DB83A
:1066D2000DC50DD80D001A0F1A1F172F183F1C4E8B
:1066E2001EE01A691E781C88189817A81AB81AC5CD
:1066F2001AD21A00250F251E212D233C254B285C7A
:106702002B6C287C258A239921A825B825CB25E046
:106712002500300E301D2C2B2E393048325C35705E
:10672200327E308D2E9B2CA930B830D230003A0EFA
:106732003A223A3D3D534064407A3D953AAA3AB8EE
:106742003AC53AD23AE03A040404040404040404C4
:1067520004040404040404040404040404040404F7
:1067620004040404040404040404040404040404E7
:1067720004040404040404040404040404040404D7
:1067820004040404040404040404040404040404C7
:0E6792000404040404040404040404040404C1
:00000001FF
